 resumethrdlst001

 Timestamp is 1fdc139a (reproducible build file hash)

 Preferred load address is 0000000180000000

 Start         Length     Name                   Class
 0001:00000000 00004110H .text$mn                CODE
 0001:00004110 00000036H .text$mn$00             CODE
 0001:00004146 00000092H .text$x                 CODE
 0002:00000000 000001d8H .idata$5                DATA
 0002:000001d8 00000038H .00cfg                  DATA
 0002:00000210 00000008H .CRT$XCA                DATA
 0002:00000218 00000008H .CRT$XCZ                DATA
 0002:00000220 00000008H .CRT$XIA                DATA
 0002:00000228 00000008H .CRT$XIC                DATA
 0002:00000230 00000008H .CRT$XIZ                DATA
 0002:00000238 00000008H .CRT$XLA                DATA
 0002:00000240 00000008H .CRT$XLZ                DATA
 0002:00000248 00000008H .CRT$XPA                DATA
 0002:00000250 00000008H .CRT$XPZ                DATA
 0002:00000258 00000008H .CRT$XTA                DATA
 0002:00000260 00000010H .CRT$XTZ                DATA
 0002:00000268 00000000H .gehcont$y              DATA
 0002:00000268 00000000H .gfids$y                DATA
 0002:00000270 00002610H .rdata                  DATA
 0002:00002880 00000000H .rdata$CastGuardVftablesA DATA
 0002:00002880 00000000H .rdata$CastGuardVftablesC DATA
 0002:00002880 00000028H .rdata$T                DATA
 0002:000028a8 000000f8H .rdata$voltmd           DATA
 0002:000029a0 00000320H .rdata$zzzdbg           DATA
 0002:00002cc0 00000008H .rtc$IAA                DATA
 0002:00002cc8 00000008H .rtc$IZZ                DATA
 0002:00002cd0 00000008H .rtc$TAA                DATA
 0002:00002cd8 00000008H .rtc$TZZ                DATA
 0002:00002ce0 00000004H .tls                    DATA
 0002:00002ce4 00000004H .tls$                   DATA
 0002:00002ce8 00000008H .tls$ZZZ                DATA
 0002:00002cf0 00000360H .xdata                  DATA
 0002:00003050 00000368H .edata                  DATA
 0002:000033b8 0000008cH .idata$2                DATA
 0002:00003444 00000014H .idata$3                DATA
 0002:00003458 000001d8H .idata$4                DATA
 0002:00003630 0000049aH .idata$6                DATA
 0003:00000000 00000080H .data                   DATA
 0003:00000080 0001b368H .bss                    DATA
 0004:00000000 000003d8H .pdata                  DATA

  Address         Publics by Value              Rva+Base               Lib:Object

 0000:00000000       __AbsoluteZero             0000000000000000     <absolute>
 0000:00000000       ___safe_se_handler_count   0000000000000000     <absolute>
 0000:00000000       ___safe_se_handler_table   0000000000000000     <absolute>
 0000:00000000       __arm64x_extra_rfe_table   0000000000000000     <absolute>
 0000:00000000       __arm64x_extra_rfe_table_size 0000000000000000     <absolute>
 0000:00000000       __arm64x_native_entrypoint 0000000000000000     <absolute>
 0000:00000000       __arm64x_redirection_metadata 0000000000000000     <absolute>
 0000:00000000       __arm64x_redirection_metadata_count 0000000000000000     <absolute>
 0000:00000000       __dynamic_value_reloc_table 0000000000000000     <absolute>
 0000:00000000       __enclave_config           0000000000000000     <absolute>
 0000:00000000       __guard_check_icall_a64n_fptr 0000000000000000     <absolute>
 0000:00000000       __guard_eh_cont_count      0000000000000000     <absolute>
 0000:00000000       __guard_eh_cont_table      0000000000000000     <absolute>
 0000:00000000       __guard_fids_count         0000000000000000     <absolute>
 0000:00000000       __guard_fids_table         0000000000000000     <absolute>
 0000:00000000       __guard_iat_count          0000000000000000     <absolute>
 0000:00000000       __guard_iat_table          0000000000000000     <absolute>
 0000:00000000       __guard_longjmp_count      0000000000000000     <absolute>
 0000:00000000       __guard_longjmp_table      0000000000000000     <absolute>
 0000:00000000       __hybrid_auxiliary_iat     0000000000000000     <absolute>
 0000:00000000       __hybrid_auxiliary_iat_copy 0000000000000000     <absolute>
 0000:00000000       __hybrid_code_map          0000000000000000     <absolute>
 0000:00000000       __hybrid_code_map_count    0000000000000000     <absolute>
 0000:00000000       __x64_code_ranges_to_entry_points 0000000000000000     <absolute>
 0000:00000000       __x64_code_ranges_to_entry_points_count 0000000000000000     <absolute>
 0000:00000100       __guard_flags              0000000000000100     <absolute>
 0000:00000000       __ImageBase                0000000180000000     <linker-defined>
 0001:00000000       ?NewObject@JNIEnv_@@QEAAPEAV_jobject@@PEAV_jclass@@PEAU_jmethodID@@ZZ 0000000180001000 f i libresumethrdlst001.obj
 0001:00000024       ?TranslateError@@YAPEBDW4jvmtiError@@@Z 0000000180001024 f   libresumethrdlst001.obj
 0001:000002dc       ?nsk_jni_check_exception@@YAHPEAUJNIEnv_@@QEBDH@Z 00000001800012dc f   libresumethrdlst001.obj
 0001:00000420       ?nsk_jni_lverify@@YAHHPEAUJNIEnv_@@HQEBDH1ZZ 0000000180001420 f   libresumethrdlst001.obj
 0001:000004c0       Agent_Initialize           00000001800014c0 f   libresumethrdlst001.obj
 0001:000006f8       Agent_OnAttach             00000001800016f8 f   libresumethrdlst001.obj
 0001:000006f8       Agent_OnLoad               00000001800016f8 f   libresumethrdlst001.obj
 0001:00000700       Java_nsk_jvmti_unit_FollowReferences_FollowRefObjects_addRefToVerify 0000000180001700 f   libresumethrdlst001.obj
 0001:000008bc       Java_nsk_jvmti_unit_FollowReferences_FollowRefObjects_getTag 00000001800018bc f   libresumethrdlst001.obj
 0001:00000978       Java_nsk_jvmti_unit_FollowReferences_FollowRefObjects_resetRefsToVerify 0000000180001978 f   libresumethrdlst001.obj
 0001:00000980       Java_nsk_jvmti_unit_FollowReferences_FollowRefObjects_resetTags 0000000180001980 f   libresumethrdlst001.obj
 0001:000009c4       Java_nsk_jvmti_unit_FollowReferences_FollowRefObjects_setTag 00000001800019c4 f   libresumethrdlst001.obj
 0001:00000c10       Java_nsk_share_jvmti_ArgumentHandler_getAgentOptionsString 0000000180001c10 f   libresumethrdlst001.obj
 0001:00000cbc       Java_nsk_share_jvmti_DebugeeClass_checkStatus 0000000180001cbc f   libresumethrdlst001.obj
 0001:00000d44       Java_nsk_share_jvmti_DebugeeClass_resetAgentData 0000000180001d44 f   libresumethrdlst001.obj
 0001:00000da4       Java_nsk_share_jvmti_RedefineAgent_agentStatus 0000000180001da4 f   libresumethrdlst001.obj
 0001:00000db0       Java_nsk_share_jvmti_RedefineAgent_isRedefined 0000000180001db0 f   libresumethrdlst001.obj
 0001:00000dbc       Java_nsk_share_jvmti_RedefineAgent_redefineAttempted 0000000180001dbc f   libresumethrdlst001.obj
 0001:00000dc8       MA_checkStatus             0000000180001dc8 f   libresumethrdlst001.obj
 0001:00000e6c       __local_stdio_printf_options 0000000180001e6c f i libresumethrdlst001.obj
 0001:00001c9c       exitOnError                0000000180002c9c f   libresumethrdlst001.obj
 0001:000020d0       fprintf                    00000001800030d0 f i libresumethrdlst001.obj
 0001:00002114       nsk_complain               0000000180003114 f   libresumethrdlst001.obj
 0001:00002140       nsk_jvmti_createJVMTIEnv   0000000180003140 f   libresumethrdlst001.obj
 0001:00002270       nsk_jvmti_findOptionIntValue 0000000180003270 f   libresumethrdlst001.obj
 0001:0000230c       nsk_jvmti_findOptionValue  000000018000330c f   libresumethrdlst001.obj
 0001:00002384       nsk_jvmti_lverify          0000000180003384 f   libresumethrdlst001.obj
 0001:00002474       nsk_jvmti_parseOptions     0000000180003474 f   libresumethrdlst001.obj
 0001:000026c4       nsk_jvmti_resetAgentData   00000001800036c4 f   libresumethrdlst001.obj
 0001:00002738       nsk_jvmti_resumeSync       0000000180003738 f   libresumethrdlst001.obj
 0001:000027dc       nsk_jvmti_waitForSync      00000001800037dc f   libresumethrdlst001.obj
 0001:000028e0       nsk_lcomplain              00000001800038e0 f   libresumethrdlst001.obj
 0001:00002900       nsk_ldisplay               0000000180003900 f   libresumethrdlst001.obj
 0001:00002920       nsk_ltrace                 0000000180003920 f   libresumethrdlst001.obj
 0001:00002940       nsk_lvcomplain             0000000180003940 f   libresumethrdlst001.obj
 0001:00002af8       nsk_lvdisplay              0000000180003af8 f   libresumethrdlst001.obj
 0001:00002b44       nsk_lverify                0000000180003b44 f   libresumethrdlst001.obj
 0001:00002ba0       nsk_lvtrace                0000000180003ba0 f   libresumethrdlst001.obj
 0001:00002c00       nsk_printf                 0000000180003c00 f   libresumethrdlst001.obj
 0001:00002c28       nsk_vprintf                0000000180003c28 f   libresumethrdlst001.obj
 0001:00002cdc       printf                     0000000180003cdc f i libresumethrdlst001.obj
 0001:000031dc       __raise_securityfailure    00000001800041dc f   MSVCRT:gs_report.obj
 0001:00003210       __report_gsfailure         0000000180004210 f   MSVCRT:gs_report.obj
 0001:00003450       __GSHandlerCheck           0000000180004450 f   MSVCRT:gshandler.obj
 0001:00003470       __GSHandlerCheckCommon     0000000180004470 f   MSVCRT:gshandler.obj
 0001:000034e0       __security_check_cookie    00000001800044e0 f   MSVCRT:amdsecgs.obj
 0001:00003820       _DllMainCRTStartup         0000000180004820 f   MSVCRT:dll_dllmain.obj
 0001:00003860       __scrt_acquire_startup_lock 0000000180004860 f   MSVCRT:utility.obj
 0001:0000389c       __scrt_dllmain_after_initialize_c 000000018000489c f   MSVCRT:utility.obj
 0001:000038d0       __scrt_dllmain_before_initialize_c 00000001800048d0 f   MSVCRT:utility.obj
 0001:000038e8       __scrt_dllmain_crt_thread_attach 00000001800048e8 f   MSVCRT:utility.obj
 0001:00003910       __scrt_dllmain_crt_thread_detach 0000000180004910 f   MSVCRT:utility.obj
 0001:00003928       __scrt_dllmain_exception_filter 0000000180004928 f   MSVCRT:utility.obj
 0001:00003988       __scrt_dllmain_uninitialize_c 0000000180004988 f   MSVCRT:utility.obj
 0001:000039b8       __scrt_dllmain_uninitialize_critical 00000001800049b8 f   MSVCRT:utility.obj
 0001:000039cc       __scrt_initialize_crt      00000001800049cc f   MSVCRT:utility.obj
 0001:00003a18       __scrt_initialize_onexit_tables 0000000180004a18 f   MSVCRT:utility.obj
 0001:00003aa4       __scrt_is_nonwritable_in_current_image 0000000180004aa4 f   MSVCRT:utility.obj
 0001:00003b3c       __scrt_release_startup_lock 0000000180004b3c f   MSVCRT:utility.obj
 0001:00003b60       __scrt_uninitialize_crt    0000000180004b60 f   MSVCRT:utility.obj
 0001:00003b8c       _onexit                    0000000180004b8c f   MSVCRT:utility.obj
 0001:00003bc8       atexit                     0000000180004bc8 f   MSVCRT:utility.obj
 0001:00003be0       __crt_debugger_hook        0000000180004be0 f   MSVCRT:utility_desktop.obj
 0001:00003be8       __scrt_fastfail            0000000180004be8 f   MSVCRT:utility_desktop.obj
 0001:00003d34       _guard_check_icall_nop     0000000180004d34 f i MSVCRT:guard_support.obj
 0001:00003d38       __security_init_cookie     0000000180004d38 f   MSVCRT:gs_support.obj
 0001:00003de4       DllMain                    0000000180004de4 f   MSVCRT:dll_dllmain_stub.obj
 0001:00003e08       ?__scrt_initialize_type_info@@YAXXZ 0000000180004e08 f   MSVCRT:tncleanup.obj
 0001:00003e18       ?__scrt_uninitialize_type_info@@YAXXZ 0000000180004e18 f   MSVCRT:tncleanup.obj
 0001:00003e24       __local_stdio_scanf_options 0000000180004e24 f i MSVCRT:default_local_stdio_options.obj
 0001:00003e2c       __scrt_initialize_default_local_stdio_options 0000000180004e2c f   MSVCRT:default_local_stdio_options.obj
 0001:00003e48       __scrt_get_dyn_tls_init_callback 0000000180004e48 f   MSVCRT:dyn_tls_init.obj
 0001:00003e50       _RTC_Initialize            0000000180004e50 f   MSVCRT:initsect.obj
 0001:00003e8c       _RTC_Terminate             0000000180004e8c f   MSVCRT:initsect.obj
 0001:00003ec8       __isa_available_init       0000000180004ec8 f   MSVCRT:cpu_disp.obj
 0001:00004074       _get_startup_argv_mode     0000000180005074 f   MSVCRT:argv_mode.obj
 0001:0000407c       __scrt_is_ucrt_dll_in_use  000000018000507c f   MSVCRT:ucrt_detection.obj
 0001:00004090       memcpy                     0000000180005090 f   vcruntime:VCRUNTIME140.dll
 0001:00004096       memset                     0000000180005096 f   vcruntime:VCRUNTIME140.dll
 0001:0000409c       strchr                     000000018000509c f   vcruntime:VCRUNTIME140.dll
 0001:000040a2       __C_specific_handler       00000001800050a2 f   vcruntime:VCRUNTIME140.dll
 0001:000040a8       __std_type_info_destroy_list 00000001800050a8 f   vcruntime:VCRUNTIME140.dll
 0001:000040ae       strcat                     00000001800050ae f   ucrt:api-ms-win-crt-string-l1-1-0.dll
 0001:000040b4       strcmp                     00000001800050b4 f   ucrt:api-ms-win-crt-string-l1-1-0.dll
 0001:000040ba       strlen                     00000001800050ba f   ucrt:api-ms-win-crt-string-l1-1-0.dll
 0001:000040c0       _initterm                  00000001800050c0 f   ucrt:api-ms-win-crt-runtime-l1-1-0.dll
 0001:000040c6       _initterm_e                00000001800050c6 f   ucrt:api-ms-win-crt-runtime-l1-1-0.dll
 0001:000040cc       _seh_filter_dll            00000001800050cc f   ucrt:api-ms-win-crt-runtime-l1-1-0.dll
 0001:000040d2       _configure_narrow_argv     00000001800050d2 f   ucrt:api-ms-win-crt-runtime-l1-1-0.dll
 0001:000040d8       _initialize_narrow_environment 00000001800050d8 f   ucrt:api-ms-win-crt-runtime-l1-1-0.dll
 0001:000040de       _initialize_onexit_table   00000001800050de f   ucrt:api-ms-win-crt-runtime-l1-1-0.dll
 0001:000040e4       _register_onexit_function  00000001800050e4 f   ucrt:api-ms-win-crt-runtime-l1-1-0.dll
 0001:000040ea       _execute_onexit_table      00000001800050ea f   ucrt:api-ms-win-crt-runtime-l1-1-0.dll
 0001:000040f0       _crt_atexit                00000001800050f0 f   ucrt:api-ms-win-crt-runtime-l1-1-0.dll
 0001:000040f6       _cexit                     00000001800050f6 f   ucrt:api-ms-win-crt-runtime-l1-1-0.dll
 0001:000040fc       __acrt_initialize          00000001800050fc f   MSVCRT:ucrt_stubs.obj
 0001:000040fc       __acrt_thread_attach       00000001800050fc f   MSVCRT:ucrt_stubs.obj
 0001:000040fc       __acrt_thread_detach       00000001800050fc f   MSVCRT:ucrt_stubs.obj
 0001:000040fc       __acrt_uninitialize        00000001800050fc f   MSVCRT:ucrt_stubs.obj
 0001:000040fc       __acrt_uninitialize_critical 00000001800050fc f   MSVCRT:ucrt_stubs.obj
 0001:000040fc       __scrt_stub_for_acrt_initialize 00000001800050fc f   MSVCRT:ucrt_stubs.obj
 0001:000040fc       __scrt_stub_for_acrt_thread_attach 00000001800050fc f   MSVCRT:ucrt_stubs.obj
 0001:000040fc       __scrt_stub_for_acrt_thread_detach 00000001800050fc f   MSVCRT:ucrt_stubs.obj
 0001:000040fc       __scrt_stub_for_acrt_uninitialize 00000001800050fc f   MSVCRT:ucrt_stubs.obj
 0001:000040fc       __scrt_stub_for_acrt_uninitialize_critical 00000001800050fc f   MSVCRT:ucrt_stubs.obj
 0001:000040fc       __vcrt_initialize          00000001800050fc f   MSVCRT:ucrt_stubs.obj
 0001:000040fc       __vcrt_thread_attach       00000001800050fc f   MSVCRT:ucrt_stubs.obj
 0001:000040fc       __vcrt_thread_detach       00000001800050fc f   MSVCRT:ucrt_stubs.obj
 0001:000040fc       __vcrt_uninitialize        00000001800050fc f   MSVCRT:ucrt_stubs.obj
 0001:000040fc       __vcrt_uninitialize_critical 00000001800050fc f   MSVCRT:ucrt_stubs.obj
 0001:00004100       __scrt_stub_for_is_c_termination_complete 0000000180005100 f   MSVCRT:ucrt_stubs.obj
 0001:00004100       _is_c_termination_complete 0000000180005100 f   MSVCRT:ucrt_stubs.obj
 0001:00004120       _guard_dispatch_icall_nop  0000000180005120 f   MSVCRT:guard_dispatch.obj
 0001:00004140       _guard_xfg_dispatch_icall_nop 0000000180005140 f   MSVCRT:guard_xfg_dispatch.obj
 0002:00000000       __imp_RtlCaptureContext    0000000180006000     kernel32:KERNEL32.dll
 0002:00000008       __imp_RtlLookupFunctionEntry 0000000180006008     kernel32:KERNEL32.dll
 0002:00000010       __imp_RtlVirtualUnwind     0000000180006010     kernel32:KERNEL32.dll
 0002:00000018       __imp_UnhandledExceptionFilter 0000000180006018     kernel32:KERNEL32.dll
 0002:00000020       __imp_SetUnhandledExceptionFilter 0000000180006020     kernel32:KERNEL32.dll
 0002:00000028       __imp_GetCurrentProcess    0000000180006028     kernel32:KERNEL32.dll
 0002:00000030       __imp_TerminateProcess     0000000180006030     kernel32:KERNEL32.dll
 0002:00000038       __imp_IsProcessorFeaturePresent 0000000180006038     kernel32:KERNEL32.dll
 0002:00000040       __imp_CloseHandle          0000000180006040     kernel32:KERNEL32.dll
 0002:00000048       __imp_InitializeCriticalSectionAndSpinCount 0000000180006048     kernel32:KERNEL32.dll
 0002:00000050       __imp_DeleteCriticalSection 0000000180006050     kernel32:KERNEL32.dll
 0002:00000058       __imp_CreateEventW         0000000180006058     kernel32:KERNEL32.dll
 0002:00000060       __imp_GetModuleHandleW     0000000180006060     kernel32:KERNEL32.dll
 0002:00000068       __imp_GetProcAddress       0000000180006068     kernel32:KERNEL32.dll
 0002:00000070       __imp_IsDebuggerPresent    0000000180006070     kernel32:KERNEL32.dll
 0002:00000078       __imp_QueryPerformanceCounter 0000000180006078     kernel32:KERNEL32.dll
 0002:00000080       __imp_GetCurrentProcessId  0000000180006080     kernel32:KERNEL32.dll
 0002:00000088       __imp_GetCurrentThreadId   0000000180006088     kernel32:KERNEL32.dll
 0002:00000090       __imp_GetSystemTimeAsFileTime 0000000180006090     kernel32:KERNEL32.dll
 0002:00000098       __imp_DisableThreadLibraryCalls 0000000180006098     kernel32:KERNEL32.dll
 0002:000000a0       __imp_InitializeSListHead  00000001800060a0     kernel32:KERNEL32.dll
 0002:000000a8       \177KERNEL32_NULL_THUNK_DATA 00000001800060a8     kernel32:KERNEL32.dll
 0002:000000b0       __imp_memcpy               00000001800060b0     vcruntime:VCRUNTIME140.dll
 0002:000000b8       __imp_memset               00000001800060b8     vcruntime:VCRUNTIME140.dll
 0002:000000c0       __imp_strchr               00000001800060c0     vcruntime:VCRUNTIME140.dll
 0002:000000c8       __imp___C_specific_handler 00000001800060c8     vcruntime:VCRUNTIME140.dll
 0002:000000d0       __imp___std_type_info_destroy_list 00000001800060d0     vcruntime:VCRUNTIME140.dll
 0002:000000d8       \177VCRUNTIME140_NULL_THUNK_DATA 00000001800060d8     vcruntime:VCRUNTIME140.dll
 0002:000000e0       __imp_strtol               00000001800060e0     ucrt:api-ms-win-crt-convert-l1-1-0.dll
 0002:000000e8       \177api-ms-win-crt-convert-l1-1-0_NULL_THUNK_DATA 00000001800060e8     ucrt:api-ms-win-crt-convert-l1-1-0.dll
 0002:000000f0       __imp_malloc               00000001800060f0     ucrt:api-ms-win-crt-heap-l1-1-0.dll
 0002:000000f8       __imp_free                 00000001800060f8     ucrt:api-ms-win-crt-heap-l1-1-0.dll
 0002:00000100       \177api-ms-win-crt-heap-l1-1-0_NULL_THUNK_DATA 0000000180006100     ucrt:api-ms-win-crt-heap-l1-1-0.dll
 0002:00000108       __imp__errno               0000000180006108     ucrt:api-ms-win-crt-runtime-l1-1-0.dll
 0002:00000110       __imp_exit                 0000000180006110     ucrt:api-ms-win-crt-runtime-l1-1-0.dll
 0002:00000118       __imp__cexit               0000000180006118     ucrt:api-ms-win-crt-runtime-l1-1-0.dll
 0002:00000120       __imp__crt_atexit          0000000180006120     ucrt:api-ms-win-crt-runtime-l1-1-0.dll
 0002:00000128       __imp__execute_onexit_table 0000000180006128     ucrt:api-ms-win-crt-runtime-l1-1-0.dll
 0002:00000130       __imp__register_onexit_function 0000000180006130     ucrt:api-ms-win-crt-runtime-l1-1-0.dll
 0002:00000138       __imp__initialize_onexit_table 0000000180006138     ucrt:api-ms-win-crt-runtime-l1-1-0.dll
 0002:00000140       __imp__initialize_narrow_environment 0000000180006140     ucrt:api-ms-win-crt-runtime-l1-1-0.dll
 0002:00000148       __imp__configure_narrow_argv 0000000180006148     ucrt:api-ms-win-crt-runtime-l1-1-0.dll
 0002:00000150       __imp__seh_filter_dll      0000000180006150     ucrt:api-ms-win-crt-runtime-l1-1-0.dll
 0002:00000158       __imp__initterm_e          0000000180006158     ucrt:api-ms-win-crt-runtime-l1-1-0.dll
 0002:00000160       __imp__initterm            0000000180006160     ucrt:api-ms-win-crt-runtime-l1-1-0.dll
 0002:00000168       \177api-ms-win-crt-runtime-l1-1-0_NULL_THUNK_DATA 0000000180006168     ucrt:api-ms-win-crt-runtime-l1-1-0.dll
 0002:00000170       __imp___acrt_iob_func      0000000180006170     ucrt:api-ms-win-crt-stdio-l1-1-0.dll
 0002:00000178       __imp_fflush               0000000180006178     ucrt:api-ms-win-crt-stdio-l1-1-0.dll
 0002:00000180       __imp___stdio_common_vsprintf 0000000180006180     ucrt:api-ms-win-crt-stdio-l1-1-0.dll
 0002:00000188       __imp___stdio_common_vfprintf 0000000180006188     ucrt:api-ms-win-crt-stdio-l1-1-0.dll
 0002:00000190       \177api-ms-win-crt-stdio-l1-1-0_NULL_THUNK_DATA 0000000180006190     ucrt:api-ms-win-crt-stdio-l1-1-0.dll
 0002:00000198       __imp_strcat               0000000180006198     ucrt:api-ms-win-crt-string-l1-1-0.dll
 0002:000001a0       __imp_strcmp               00000001800061a0     ucrt:api-ms-win-crt-string-l1-1-0.dll
 0002:000001a8       __imp__strdup              00000001800061a8     ucrt:api-ms-win-crt-string-l1-1-0.dll
 0002:000001a8       __imp_strdup               00000001800061a8     ucrt:api-ms-win-crt-string-l1-1-0.dll
 0002:000001b0       __imp_strlen               00000001800061b0     ucrt:api-ms-win-crt-string-l1-1-0.dll
 0002:000001b8       __imp_strncmp              00000001800061b8     ucrt:api-ms-win-crt-string-l1-1-0.dll
 0002:000001c0       __imp_strpbrk              00000001800061c0     ucrt:api-ms-win-crt-string-l1-1-0.dll
 0002:000001c8       __imp_strncpy              00000001800061c8     ucrt:api-ms-win-crt-string-l1-1-0.dll
 0002:000001d0       \177api-ms-win-crt-string-l1-1-0_NULL_THUNK_DATA 00000001800061d0     ucrt:api-ms-win-crt-string-l1-1-0.dll
 0002:000001d8       __guard_check_icall_fptr   00000001800061d8     MSVCRT:guard_support.obj
 0002:000001e0       __guard_xfg_check_icall_fptr 00000001800061e0     MSVCRT:guard_support.obj
 0002:000001e8       __guard_dispatch_icall_fptr 00000001800061e8     MSVCRT:guard_support.obj
 0002:000001f0       __guard_xfg_dispatch_icall_fptr 00000001800061f0     MSVCRT:guard_support.obj
 0002:000001f8       __guard_xfg_table_dispatch_icall_fptr 00000001800061f8     MSVCRT:guard_support.obj
 0002:00000200       __castguard_check_failure_os_handled_fptr 0000000180006200     MSVCRT:guard_support.obj
 0002:00000208       __guard_memcpy_fptr        0000000180006208     vcruntime:softmemtag.obj
 0002:00000210       __xc_a                     0000000180006210     MSVCRT:initializers.obj
 0002:00000218       __xc_z                     0000000180006218     MSVCRT:initializers.obj
 0002:00000220       __xi_a                     0000000180006220     MSVCRT:initializers.obj
 0002:00000230       __xi_z                     0000000180006230     MSVCRT:initializers.obj
 0002:00000238       __xl_a                     0000000180006238     MSVCRT:tlssup.obj
 0002:00000240       __xl_z                     0000000180006240     MSVCRT:tlssup.obj
 0002:00000248       __xp_a                     0000000180006248     MSVCRT:initializers.obj
 0002:00000250       __xp_z                     0000000180006250     MSVCRT:initializers.obj
 0002:00000258       __xt_a                     0000000180006258     MSVCRT:initializers.obj
 0002:00000260       __xt_z                     0000000180006260     MSVCRT:initializers.obj
 0002:00000270       g_refKindStr               0000000180006270     libresumethrdlst001.obj
 0002:00000420       ??_C@_09BPLDFGCI@unknown_0@ 0000000180006420     libresumethrdlst001.obj
 0002:00000430       ??_C@_0BL@FPNMECJD@JVMTI_HEAP_REFERENCE_CLASS@ 0000000180006430     libresumethrdlst001.obj
 0002:00000450       ??_C@_0BL@FKGKKLNM@JVMTI_HEAP_REFERENCE_FIELD@ 0000000180006450     libresumethrdlst001.obj
 0002:00000470       ??_C@_0CD@CAEHCFJF@JVMTI_HEAP_REFERENCE_ARRAY_ELEM@ 0000000180006470     libresumethrdlst001.obj
 0002:00000498       ??_C@_0CC@DNEBMCNK@JVMTI_HEAP_REFERENCE_CLASS_LOAD@ 0000000180006498     libresumethrdlst001.obj
 0002:000004c0       ??_C@_0BN@CJMIPEBB@JVMTI_HEAP_REFERENCE_SIGNERS@ 00000001800064c0     libresumethrdlst001.obj
 0002:000004e0       ??_C@_0CH@HBOIDPEB@JVMTI_HEAP_REFERENCE_PROTECTION@ 00000001800064e0     libresumethrdlst001.obj
 0002:00000508       ??_C@_0BP@MDKGDGKL@JVMTI_HEAP_REFERENCE_INTERFACE@ 0000000180006508     libresumethrdlst001.obj
 0002:00000528       ??_C@_0CC@JJMIHNJH@JVMTI_HEAP_REFERENCE_STATIC_FIE@ 0000000180006528     libresumethrdlst001.obj
 0002:00000550       ??_C@_0CD@IDHEEGID@JVMTI_HEAP_REFERENCE_CONSTANT_P@ 0000000180006550     libresumethrdlst001.obj
 0002:00000578       ??_C@_0CA@EFFCHNG@JVMTI_HEAP_REFERENCE_SUPERCLASS@ 0000000180006578     libresumethrdlst001.obj
 0002:00000598       ??_C@_0L@PCDFHGCJ@unknown_11@ 0000000180006598     libresumethrdlst001.obj
 0002:000005a8       ??_C@_0L@NJBICFOK@unknown_12@ 00000001800065a8     libresumethrdlst001.obj
 0002:000005b8       ??_C@_0L@MAADBEKL@unknown_13@ 00000001800065b8     libresumethrdlst001.obj
 0002:000005c8       ??_C@_0L@IPECICGM@unknown_14@ 00000001800065c8     libresumethrdlst001.obj
 0002:000005d8       ??_C@_0L@JGFJLDCN@unknown_15@ 00000001800065d8     libresumethrdlst001.obj
 0002:000005e8       ??_C@_0L@LNHEOAOO@unknown_16@ 00000001800065e8     libresumethrdlst001.obj
 0002:000005f8       ??_C@_0L@KEGPNBKP@unknown_17@ 00000001800065f8     libresumethrdlst001.obj
 0002:00000608       ??_C@_0L@CDPHMNGA@unknown_18@ 0000000180006608     libresumethrdlst001.obj
 0002:00000618       ??_C@_0L@DKOMPMCB@unknown_19@ 0000000180006618     libresumethrdlst001.obj
 0002:00000628       ??_C@_0L@OJGIPJDB@unknown_20@ 0000000180006628     libresumethrdlst001.obj
 0002:00000638       ??_C@_0CA@KAOFNDEM@JVMTI_HEAP_REFERENCE_JNI_GLOBAL@ 0000000180006638     libresumethrdlst001.obj
 0002:00000658       ??_C@_0CC@HPFAJBK@JVMTI_HEAP_REFERENCE_SYSTEM_CLA@ 0000000180006658     libresumethrdlst001.obj
 0002:00000680       ??_C@_0BN@FDEGFOHC@JVMTI_HEAP_REFERENCE_MONITOR@ 0000000180006680     libresumethrdlst001.obj
 0002:000006a0       ??_C@_0CB@HKIBCMAJ@JVMTI_HEAP_REFERENCE_STACK_LOCA@ 00000001800066a0     libresumethrdlst001.obj
 0002:000006c8       ??_C@_0BP@EAACMMOE@JVMTI_HEAP_REFERENCE_JNI_LOCAL@ 00000001800066c8     libresumethrdlst001.obj
 0002:000006e8       ??_C@_0BM@IJDEOGOE@JVMTI_HEAP_REFERENCE_THREAD@ 00000001800066e8     libresumethrdlst001.obj
 0002:00000708       ??_C@_0BL@EDGPPKC@JVMTI_HEAP_REFERENCE_OTHER@ 0000000180006708     libresumethrdlst001.obj
 0002:00000724       ??_C@_04BCJPDBDA@Code@     0000000180006724     libresumethrdlst001.obj
 0002:00000730       ??_C@_0BA@OCLMCFKC@LineNumberTable@ 0000000180006730     libresumethrdlst001.obj
 0002:00000740       ??_C@_0BD@CPAEPILC@LocalVariableTable@ 0000000180006740     libresumethrdlst001.obj
 0002:00000758       ??_C@_0BH@NMBDNHBD@LocalVariableTypeTable@ 0000000180006758     libresumethrdlst001.obj
 0002:00000770       ??_C@_0O@HIHEEDNJ@StackMapTable@ 0000000180006770     libresumethrdlst001.obj
 0002:00000780       ??_C@_0L@HCDIAMJG@?9?5?$CFs?0?5?$CFd?3?5@ 0000000180006780     libresumethrdlst001.obj
 0002:00000790       ??_C@_0JI@HLPECLFI@?$CD?5?4?4?4?6?$CD?5ERROR?3?5too?5many?5complai@ 0000000180006790     libresumethrdlst001.obj
 0002:00000830       ??_C@_0ED@JNEKCCOB@The?5following?5fake?5exception?5st@ 0000000180006830     libresumethrdlst001.obj
 0002:00000878       ??_C@_0CN@FCNMDFBH@nsk?4share?4Fake_Exception_for_RU@ 0000000180006878     libresumethrdlst001.obj
 0002:000008a8       ??_C@_08PGFFNAEI@?$CI?$CFs?3?$CFd?$CJ?5@ 00000001800068a8     libresumethrdlst001.obj
 0002:000008b8       ??_C@_0DP@IENMAEGI@s?2test?2hotspot?2jtreg?2vmTestbase@ 00000001800068b8     libresumethrdlst001.obj
 0002:000008f8       ??_C@_0BL@NDJLFFJB@?7at?5nsk_lvcomplain?$CI?$CFs?3?$CFd?$CJ?6@ 00000001800068f8     libresumethrdlst001.obj
 0002:00000918       ??_C@_0BC@JOOKAFKF@?$CD?5ERROR?3?5?$CFs?0?5?$CFd?3?5@ 0000000180006918     libresumethrdlst001.obj
 0002:00000930       ??_C@_09KJEAHMEH@?$CD?5ERROR?3?5@ 0000000180006930     libresumethrdlst001.obj
 0002:0000093c       ??_C@_02GPIOPFAK@?$DO?$DO@ 000000018000693c     libresumethrdlst001.obj
 0002:00000940       ??_C@_02FODMEDOG@?$DM?$DM@ 0000000180006940     libresumethrdlst001.obj
 0002:00000944       ??_C@_02DJGKEECL@?4?4@     0000000180006944     libresumethrdlst001.obj
 0002:00000948       ??_C@_0O@CJPGJOAF@?9?5?$CFs?0?5?$CFd?3?5?$CFs?5@ 0000000180006948     libresumethrdlst001.obj
 0002:00000958       ??_C@_0CB@IAKPDOIC@?$CD?5?5?5verified?5assertion?5is?5FALSE@ 0000000180006958     libresumethrdlst001.obj
 0002:00000980       ??_C@_0CO@LGONDEPD@stdout?3?5fflush?5failed?5?9?5err?$DN?$CFd?5@ 0000000180006980     libresumethrdlst001.obj
 0002:000009b0       ??_C@_0CO@KBGKJPBD@stderr?3?5fflush?5failed?5?9?5err?$DN?$CFd?5@ 00000001800069b0     libresumethrdlst001.obj
 0002:000009e0       ??_C@_06PAOMPDJH@?$DMnone?$DO@ 00000001800069e0     libresumethrdlst001.obj
 0002:000009e8       ??_C@_06PHAKILGJ@?5ALIVE@  00000001800069e8     libresumethrdlst001.obj
 0002:000009f0       ??_C@_0M@OFKKEJHG@?5TERMINATED@ 00000001800069f0     libresumethrdlst001.obj
 0002:00000a00       ??_C@_09JDCMELJI@?5RUNNABLE@ 0000000180006a00     libresumethrdlst001.obj
 0002:00000a10       ??_C@_08OAHMLBPA@?5WAITING@ 0000000180006a10     libresumethrdlst001.obj
 0002:00000a20       ??_C@_0BG@GOEBACGE@?5WAITING_INDEFINITELY@ 0000000180006a20     libresumethrdlst001.obj
 0002:00000a38       ??_C@_0BG@CCLPBKFG@?5WAITING_WITH_TIMEOUT@ 0000000180006a38     libresumethrdlst001.obj
 0002:00000a50       ??_C@_09DEFAFODN@?5SLEEPING@ 0000000180006a50     libresumethrdlst001.obj
 0002:00000a60       ??_C@_0BA@EIDDAKGK@?5IN_OBJECT_WAIT@ 0000000180006a60     libresumethrdlst001.obj
 0002:00000a70       ??_C@_07GIPIPEAD@?5PARKED@ 0000000180006a70     libresumethrdlst001.obj
 0002:00000a78       ??_C@_0BK@LNIHGEJF@?5BLOCKED_ON_MONITOR_ENTER@ 0000000180006a78     libresumethrdlst001.obj
 0002:00000a98       ??_C@_0L@MOBKJCJD@?5SUSPENDED@ 0000000180006a98     libresumethrdlst001.obj
 0002:00000aa8       ??_C@_0N@CPMJCKAP@?5INTERRUPTED@ 0000000180006aa8     libresumethrdlst001.obj
 0002:00000ab8       ??_C@_0L@PEJNJEEC@?5IN_NATIVE@ 0000000180006ab8     libresumethrdlst001.obj
 0002:00000ac8       ??_C@_0BB@JCNMKLLK@JVMTI_ERROR_NONE@ 0000000180006ac8     libresumethrdlst001.obj
 0002:00000ae0       ??_C@_0BL@LDIMKLPH@JVMTI_ERROR_INVALID_THREAD@ 0000000180006ae0     libresumethrdlst001.obj
 0002:00000b00       ??_C@_0CB@PJFPAIKJ@JVMTI_ERROR_INVALID_THREAD_GROU@ 0000000180006b00     libresumethrdlst001.obj
 0002:00000b28       ??_C@_0BN@LLMKHMNF@JVMTI_ERROR_INVALID_PRIORITY@ 0000000180006b28     libresumethrdlst001.obj
 0002:00000b48       ??_C@_0CB@MBOFKAGB@JVMTI_ERROR_THREAD_NOT_SUSPENDE@ 0000000180006b48     libresumethrdlst001.obj
 0002:00000b70       ??_C@_0BN@FABOLPBI@JVMTI_ERROR_THREAD_SUSPENDED@ 0000000180006b70     libresumethrdlst001.obj
 0002:00000b90       ??_C@_0BN@FDGNOBJM@JVMTI_ERROR_THREAD_NOT_ALIVE@ 0000000180006b90     libresumethrdlst001.obj
 0002:00000bb0       ??_C@_0BL@GOBIFKNJ@JVMTI_ERROR_INVALID_OBJECT@ 0000000180006bb0     libresumethrdlst001.obj
 0002:00000bd0       ??_C@_0BK@FCMAJPPC@JVMTI_ERROR_INVALID_CLASS@ 0000000180006bd0     libresumethrdlst001.obj
 0002:00000bf0       ??_C@_0BP@IKLLBKEB@JVMTI_ERROR_CLASS_NOT_PREPARED@ 0000000180006bf0     libresumethrdlst001.obj
 0002:00000c10       ??_C@_0BN@KLPPLKG@JVMTI_ERROR_INVALID_METHODID@ 0000000180006c10     libresumethrdlst001.obj
 0002:00000c30       ??_C@_0BN@BCEKOKND@JVMTI_ERROR_INVALID_LOCATION@ 0000000180006c30     libresumethrdlst001.obj
 0002:00000c50       ??_C@_0BM@DFDGPME@JVMTI_ERROR_INVALID_FIELDID@ 0000000180006c50     libresumethrdlst001.obj
 0002:00000c70       ??_C@_0BL@NELIEPEC@JVMTI_ERROR_NO_MORE_FRAMES@ 0000000180006c70     libresumethrdlst001.obj
 0002:00000c90       ??_C@_0BJ@BDBECFDM@JVMTI_ERROR_OPAQUE_FRAME@ 0000000180006c90     libresumethrdlst001.obj
 0002:00000cb0       ??_C@_0BK@MIIFNLOB@JVMTI_ERROR_TYPE_MISMATCH@ 0000000180006cb0     libresumethrdlst001.obj
 0002:00000cd0       ??_C@_0BJ@HPCAOILC@JVMTI_ERROR_INVALID_SLOT@ 0000000180006cd0     libresumethrdlst001.obj
 0002:00000cf0       ??_C@_0BG@CHILOPNI@JVMTI_ERROR_DUPLICATE@ 0000000180006cf0     libresumethrdlst001.obj
 0002:00000d08       ??_C@_0BG@DIEMLHKM@JVMTI_ERROR_NOT_FOUND@ 0000000180006d08     libresumethrdlst001.obj
 0002:00000d20       ??_C@_0BM@NHMCKHOB@JVMTI_ERROR_INVALID_MONITOR@ 0000000180006d20     libresumethrdlst001.obj
 0002:00000d40       ??_C@_0BO@PPEDAJGL@JVMTI_ERROR_NOT_MONITOR_OWNER@ 0000000180006d40     libresumethrdlst001.obj
 0002:00000d60       ??_C@_0BG@FCAIPEID@JVMTI_ERROR_INTERRUPT@ 0000000180006d60     libresumethrdlst001.obj
 0002:00000d78       ??_C@_0CB@EGDBNKOI@JVMTI_ERROR_INVALID_CLASS_FORMA@ 0000000180006d78     libresumethrdlst001.obj
 0002:00000da0       ??_C@_0CG@DGKOGIAL@JVMTI_ERROR_CIRCULAR_CLASS_DEFI@ 0000000180006da0     libresumethrdlst001.obj
 0002:00000dc8       ??_C@_0BP@ICEALPKC@JVMTI_ERROR_FAILS_VERIFICATION@ 0000000180006dc8     libresumethrdlst001.obj
 0002:00000de8       ??_C@_0DC@JDACLMIO@JVMTI_ERROR_UNSUPPORTED_REDEFIN@ 0000000180006de8     libresumethrdlst001.obj
 0002:00000e20       ??_C@_0DE@GKDKNOMJ@JVMTI_ERROR_UNSUPPORTED_REDEFIN@ 0000000180006e20     libresumethrdlst001.obj
 0002:00000e58       ??_C@_0BO@LAFKIOG@JVMTI_ERROR_INVALID_TYPESTATE@ 0000000180006e58     libresumethrdlst001.obj
 0002:00000e78       ??_C@_0DH@INDGCLLB@JVMTI_ERROR_UNSUPPORTED_REDEFIN@ 0000000180006e78     libresumethrdlst001.obj
 0002:00000eb0       ??_C@_0DE@NHEOMMGI@JVMTI_ERROR_UNSUPPORTED_REDEFIN@ 0000000180006eb0     libresumethrdlst001.obj
 0002:00000ee8       ??_C@_0CA@EKPNJOEP@JVMTI_ERROR_UNSUPPORTED_VERSION@ 0000000180006ee8     libresumethrdlst001.obj
 0002:00000f08       ??_C@_0BN@OFFMAHHL@JVMTI_ERROR_NAMES_DONT_MATCH@ 0000000180006f08     libresumethrdlst001.obj
 0002:00000f28       ??_C@_0DN@HHBBLAKE@JVMTI_ERROR_UNSUPPORTED_REDEFIN@ 0000000180006f28     libresumethrdlst001.obj
 0002:00000f68       ??_C@_0DO@HMBGBGNA@JVMTI_ERROR_UNSUPPORTED_REDEFIN@ 0000000180006f68     libresumethrdlst001.obj
 0002:00000fa8       ??_C@_0BP@PBECGKHJ@JVMTI_ERROR_UNMODIFIABLE_CLASS@ 0000000180006fa8     libresumethrdlst001.obj
 0002:00000fc8       ??_C@_0BK@CANILEHF@JVMTI_ERROR_NOT_AVAILABLE@ 0000000180006fc8     libresumethrdlst001.obj
 0002:00000fe8       ??_C@_0CE@INJKMEFK@JVMTI_ERROR_MUST_POSSESS_CAPABI@ 0000000180006fe8     libresumethrdlst001.obj
 0002:00001010       ??_C@_0BJ@LBFPFPDM@JVMTI_ERROR_NULL_POINTER@ 0000000180007010     libresumethrdlst001.obj
 0002:00001030       ??_C@_0BP@CHJPNNEM@JVMTI_ERROR_ABSENT_INFORMATION@ 0000000180007030     libresumethrdlst001.obj
 0002:00001050       ??_C@_0BP@OMFMNLC@JVMTI_ERROR_INVALID_EVENT_TYPE@ 0000000180007050     libresumethrdlst001.obj
 0002:00001070       ??_C@_0BN@BIBNPHHO@JVMTI_ERROR_ILLEGAL_ARGUMENT@ 0000000180007070     libresumethrdlst001.obj
 0002:00001090       ??_C@_0BK@KKNDHDCE@JVMTI_ERROR_NATIVE_METHOD@ 0000000180007090     libresumethrdlst001.obj
 0002:000010b0       ??_C@_0BK@PMKCFHAE@JVMTI_ERROR_OUT_OF_MEMORY@ 00000001800070b0     libresumethrdlst001.obj
 0002:000010d0       ??_C@_0BK@NNJBDMNB@JVMTI_ERROR_ACCESS_DENIED@ 00000001800070d0     libresumethrdlst001.obj
 0002:000010f0       ??_C@_0BI@GHECLMNC@JVMTI_ERROR_WRONG_PHASE@ 00000001800070f0     libresumethrdlst001.obj
 0002:00001108       ??_C@_0BF@OLIHJOII@JVMTI_ERROR_INTERNAL@ 0000000180007108     libresumethrdlst001.obj
 0002:00001120       ??_C@_0BO@EOHGKJHI@JVMTI_ERROR_UNATTACHED_THREAD@ 0000000180007120     libresumethrdlst001.obj
 0002:00001140       ??_C@_0CA@LKHFDACL@JVMTI_ERROR_INVALID_ENVIRONMENT@ 0000000180007140     libresumethrdlst001.obj
 0002:00001160       ??_C@_0BA@MMFHLOKK@?$DMunknown?5error?$DO@ 0000000180007160     libresumethrdlst001.obj
 0002:00001170       ??_C@_0CF@CBHOKDB@throwable?5?$DN?5jni?9?$DOExceptionOccur@ 0000000180007170     libresumethrdlst001.obj
 0002:00001198       ??_C@_03OFAPEBGM@?$CFs?6@  0000000180007198     libresumethrdlst001.obj
 0002:000011a0       ??_C@_0DM@LPIGEGNJ@s?2test?2hotspot?2jtreg?2vmTestbase@ 00000001800071a0     libresumethrdlst001.obj
 0002:000011e0       ??_C@_0CC@NFCNPEPK@Exception?5in?5JNI?5call?5?$CIcleared?$CJ@ 00000001800071e0     libresumethrdlst001.obj
 0002:00001208       ??_C@_0BJ@IBAKFIKF@jni?9?$DOExceptionDescribe?$CI?$CJ@ 0000000180007208     libresumethrdlst001.obj
 0002:00001228       ??_C@_0BG@GGKALKMH@jni?9?$DOExceptionClear?$CI?$CJ@ 0000000180007228     libresumethrdlst001.obj
 0002:00001240       ??_C@_0CF@JMGFGJLJ@?$CD?5?5?5verified?5JNI?5assertion?5is?5F@ 0000000180007240     libresumethrdlst001.obj
 0002:00001268       ??_C@_07KBAMPNJK@verbose@  0000000180007268     libresumethrdlst001.obj
 0002:00001270       ??_C@_0DN@PKJBOLAP@nsk_jvmti_parseOptions?$CI?$CJ?3?5unexp@ 0000000180007270     libresumethrdlst001.obj
 0002:000012b0       ??_C@_05IMBNNINJ@trace@    00000001800072b0     libresumethrdlst001.obj
 0002:000012b8       ??_C@_0DD@BJKGNDMB@nsk_jvmti_parseOptions?$CI?$CJ?3?5no?5va@ 00000001800072b8     libresumethrdlst001.obj
 0002:000012ec       ??_C@_04CGFJFPFD@none@     00000001800072ec     libresumethrdlst001.obj
 0002:000012f4       ??_C@_06BMELKFMA@before@   00000001800072f4     libresumethrdlst001.obj
 0002:000012fc       ??_C@_05CMKPCFDK@after@    00000001800072fc     libresumethrdlst001.obj
 0002:00001304       ??_C@_03NFKEKGGK@all@      0000000180007304     libresumethrdlst001.obj
 0002:00001308       ??_C@_0DM@NDNJGJKE@nsk_jvmti_parseOptions?$CI?$CJ?3?5uexpe@ 0000000180007308     libresumethrdlst001.obj
 0002:00001348       ??_C@_08NBBJKJO@waittime@  0000000180007348     libresumethrdlst001.obj
 0002:00001358       ??_C@_0DO@CMHGAOHC@nsk_jvmti_parseOptions?$CI?$CJ?3?5not?5i@ 0000000180007358     libresumethrdlst001.obj
 0002:00001398       ??_C@_0DL@LNMPBDLN@nsk_jvmti_parseOptions?$CI?$CJ?3?5negat@ 0000000180007398     libresumethrdlst001.obj
 0002:000013d8       ??_C@_0DA@GMFJNOJH@nsk_jvmti_parseOptions?$CI?$CJ?3?5unkno@ 00000001800073d8     libresumethrdlst001.obj
 0002:00001408       ??_C@_0CO@CCIAMEAN@nsk_jvmti_parseOptions?$CI?$CJ?3?5found@ 0000000180007408     libresumethrdlst001.obj
 0002:00001438       ??_C@_0CJ@OEGPCGDL@nsk_jvmti_parseOptions?$CI?$CJ?3?5out?5o@ 0000000180007438     libresumethrdlst001.obj
 0002:00001468       ??_C@_0DI@NMBHPGGF@nsk_jvmti_parseOptions?$CI?$CJ?3?5too?5m@ 0000000180007468     libresumethrdlst001.obj
 0002:000014a0       ??_C@_03POGCGECB@?5?0?$HO@ 00000001800074a0     libresumethrdlst001.obj
 0002:000014a8       ??_C@_0DC@GKLNPJIJ@nsk_jvmti_findOptionValue?$CI?$CJ?3?5op@ 00000001800074a8     libresumethrdlst001.obj
 0002:000014e0       ??_C@_0DF@OPPIHBPJ@nsk_jvmti_findOptionIntValue?$CI?$CJ?3@ 00000001800074e0     libresumethrdlst001.obj
 0002:00001518       ??_C@_0DO@DBKDODPI@nsk_jvmti_findOptionIntValue?$CI?$CJ?3@ 0000000180007518     libresumethrdlst001.obj
 0002:00001560       ??_C@_0EE@NGNPKOJC@nsk_jvmti_findOptionIntValue?$CI?$CJ?3@ 0000000180007560     libresumethrdlst001.obj
 0002:000015a8       ??_C@_0CB@MLNJNCLJ@?5?5jvmti?5error?3?5code?$DN?$CFd?0?5name?$DN?$CFs@ 00000001800075a8     libresumethrdlst001.obj
 0002:000015d0       ??_C@_0CD@OHBGDKMK@?$CD?5?5?5jvmti?5error?3?5code?$DN?$CFd?0?5name?$DN@ 00000001800075d0     libresumethrdlst001.obj
 0002:000015f8       ??_C@_0CG@JNNCGPHB@?$CD?5?5?5error?5expected?3?5code?$DN?$CFd?0?5na@ 00000001800075f8     libresumethrdlst001.obj
 0002:00001620       ??_C@_0EB@IMGKPCGE@?$CIstr_obj?5?$DN?5jni?9?$DONewStringUTF?$CIco@ 0000000180007620     libresumethrdlst001.obj
 0002:00001670       ??_C@_0EA@HFOGGBCC@s?2test?2hotspot?2jtreg?2vmTestbase@ 0000000180007670     libresumethrdlst001.obj
 0002:000016b0       ??_C@_05KKCIMGE@error@     00000001800076b0     libresumethrdlst001.obj
 0002:000016b8       ??_C@_0BD@HGNAOMCP@agent_data_monitor@ 00000001800076b8     libresumethrdlst001.obj
 0002:000016d0       ??_C@_0EB@OGCLGKLN@javaVM?9?$DOGetEnv?$CI?$CIvoid?5?$CK?$CK?$CJ?$CGjvmti_@ 00000001800076d0     libresumethrdlst001.obj
 0002:00001720       ??_C@_0EA@PNBCDMOA@s?2test?2hotspot?2jtreg?2vmTestbase@ 0000000180007720     libresumethrdlst001.obj
 0002:00001760       ??_C@_0CI@DDPIFBGM@init_agent_data?$CIjvmti_env?0?5?$CGage@ 0000000180007760     libresumethrdlst001.obj
 0002:00001788       ??_C@_0DI@ILAHDLMP@?$CI?$CKagentThreadProc?$CJ?$CIjvmti_env?0?5a@ 0000000180007788     libresumethrdlst001.obj
 0002:000017c0       ??_C@_0BD@KDBALNLB@JVMTI?5agent?5thread@ 00000001800077c0     libresumethrdlst001.obj
 0002:000017d8       ??_C@_0BB@NOKBFPFO@java?1lang?1Thread@ 00000001800077d8     libresumethrdlst001.obj
 0002:000017ec       ??_C@_06FALKBLGB@?$DMinit?$DO@ 00000001800077ec     libresumethrdlst001.obj
 0002:000017f8       ??_C@_0BG@IKDDPPGD@?$CILjava?1lang?1String?$DL?$CJV@ 00000001800077f8     libresumethrdlst001.obj
 0002:00001810       ??_C@_0EB@IFJBFEKC@?$CIthreadClass?5?$DN?5jni_env?9?$DOFindCla@ 0000000180007810     libresumethrdlst001.obj
 0002:00001860       ??_C@_0GF@FGFIBKKL@?$CIthreadCtor?5?$DN?5jni_env?9?$DOGetMetho@ 0000000180007860     libresumethrdlst001.obj
 0002:000018c8       ??_C@_0DN@NCPDJLOG@?$CIthreadName?5?$DN?5jni_env?9?$DONewStrin@ 00000001800078c8     libresumethrdlst001.obj
 0002:00001910       ??_C@_0FE@PFKODBGC@?$CIthreadObject?5?$DN?5jni_env?9?$DONewObj@ 0000000180007910     libresumethrdlst001.obj
 0002:00001970       ??_C@_0ED@HOBAHHJI@?$CIthreadGlobalRef?5?$DN?5jni_env?9?$DONew@ 0000000180007970     libresumethrdlst001.obj
 0002:000019c0       ??_C@_0FN@HNJJAHFC@jvmti_env?9?$DORunAgentThread?$CIagent@ 00000001800079c0     libresumethrdlst001.obj
 0002:00001a20       ??_C@_0EA@MOJDNKDF@Debuggee?5status?5sync?5aborted?5be@ 0000000180007a20     libresumethrdlst001.obj
 0002:00001a60       ??_C@_0CO@PGPGMHBJ@No?5status?5sync?5occured?5for?5time@ 0000000180007a60     libresumethrdlst001.obj
 0002:00001a90       ??_C@_0CL@DOEBDPKJ@Debuggee?5was?5not?5suspended?5on?5s@ 0000000180007a90     libresumethrdlst001.obj
 0002:00001ac0       ??_C@_0EA@EEOEJAEN@status?5?$DN?5syncDebuggeeStatus?$CIjni@ 0000000180007ac0     libresumethrdlst001.obj
 0002:00001b00       ??_C@_0BL@JBCFNBMB@nsk_jvmti_resetAgentData?$CI?$CJ@ 0000000180007b00     libresumethrdlst001.obj
 0002:00001b20       ??_C@_0EL@LPBEELIP@s?2test?2hotspot?2jtreg?2vmTestbase@ 0000000180007b20     libresumethrdlst001.obj
 0002:00001b70       ??_C@_0CK@JDAMFDMJ@jvmti?9?$DOSetTag?$CIo?0?5tag?$CJ?5?$DN?$DN?5JVMTI_@ 0000000180007b70     libresumethrdlst001.obj
 0002:00001ba0       ??_C@_0CC@DAMNHKNI@Can?8t?5set?5tag?5?$CFli?5for?5object?5?$CFl@ 0000000180007ba0     libresumethrdlst001.obj
 0002:00001bc8       ??_C@_0DL@HAJPNKEF@jvmti?9?$DOGetObjectHashCode?$CIo?0?5?$CGha@ 0000000180007bc8     libresumethrdlst001.obj
 0002:00001c08       ??_C@_0BL@JFPIEOBF@Can?8t?5get?5hash?5object?5?$CFlx?6@ 0000000180007c08     libresumethrdlst001.obj
 0002:00001c28       ??_C@_0BG@DICPHBKN@setTag?3?5?$CF08x?5?$DM?9?5?$CF?53li@ 0000000180007c28     libresumethrdlst001.obj
 0002:00001c40       ??_C@_0DH@FCEEBDMJ@?$CIs?5?$DN?5jni?9?$DOGetStringUTFChars?$CIsIn@ 0000000180007c40     libresumethrdlst001.obj
 0002:00001c78       ??_C@_0BJ@OKKGHDCN@Can?8t?5get?5string?5at?5?$CF?$CDp?6@ 0000000180007c78     libresumethrdlst001.obj
 0002:00001c98       ??_C@_0BP@EKFLGGFJ@Can?8t?5get?5string?5at?5?$CF?$CDp?3?5null?6@ 0000000180007c98     libresumethrdlst001.obj
 0002:00001cb8       ??_C@_06ICODBHCL@?5?1?1?5?$CFs@ 0000000180007cb8     libresumethrdlst001.obj
 0002:00001cc0       ??_C@_0DB@KGFPLEGO@?$CIr?5?$DN?5jvmti?9?$DOGetTag?$CIo?0?5?$CGtag?$CJ?$CJ?5?$DN?$DN@ 0000000180007cc0     libresumethrdlst001.obj
 0002:00001cf8       ??_C@_0CO@PDAGBCGJ@Can?8t?5GetTag?5for?5object?5?$CFlx?4?5Re@ 0000000180007cf8     libresumethrdlst001.obj
 0002:00001d28       ??_C@_0CH@HPEODOHC@TEST_BUG?3?5Max?4?5number?5of?5refs?5r@ 0000000180007d28     libresumethrdlst001.obj
 0002:00001d50       ??_C@_0DI@PHFCABIM@?$CIr?5?$DN?5jvmti?9?$DOGetTag?$CIfrom?0?5?$CGtagFr@ 0000000180007d50     libresumethrdlst001.obj
 0002:00001d88       ??_C@_0DI@MDEGFNKD@TEST_BUG?3?5Can?8t?5GetTag?5for?5obje@ 0000000180007d88     libresumethrdlst001.obj
 0002:00001dc0       ??_C@_0DE@MLELJAHM@?$CIr?5?$DN?5jvmti?9?$DOGetTag?$CIto?0?5?$CGtagTo?$CJ?$CJ@ 0000000180007dc0     libresumethrdlst001.obj
 0002:00001df8       ??_C@_0BL@GFNEFEMB@Wait?5for?5threads?5to?5start?6@ 0000000180007df8     libresumethrdlst001.obj
 0002:00001e20       ??_C@_0GB@HMMIGFBF@s?2test?2hotspot?2jtreg?2vmTestbase@ 0000000180007e20     libresumethrdlst001.obj
 0002:00001e88       ??_C@_0CE@EBCICDHF@Allocate?5threads?5array?3?5?$CFd?5thre@ 0000000180007e88     libresumethrdlst001.obj
 0002:00001eb0       ??_C@_0EN@IFCLFNP@jvmti?9?$DOAllocate?$CI?$CIthreadsCount?5?$CK@ 0000000180007eb0     libresumethrdlst001.obj
 0002:00001f00       ??_C@_0BL@CADLDGMG@?5?5?4?4?4?5allocated?5array?3?5?$CFp?6@ 0000000180007f00     libresumethrdlst001.obj
 0002:00001f20       ??_C@_0CE@INFAMOFE@Allocate?5results?5array?3?5?$CFd?5thre@ 0000000180007f20     libresumethrdlst001.obj
 0002:00001f50       ??_C@_0FA@OKDDMAKC@jvmti?9?$DOAllocate?$CI?$CIthreadsCount?5?$CK@ 0000000180007f50     libresumethrdlst001.obj
 0002:00001fa0       ??_C@_0BK@EBGMDDGN@Find?5threads?3?5?$CFd?5threads?6@ 0000000180007fa0     libresumethrdlst001.obj
 0002:00001fc0       ??_C@_0EC@PKONHJMO@fillThreadsByName?$CIjvmti?0?5jni?0?5T@ 0000000180007fc0     libresumethrdlst001.obj
 0002:00002008       ??_C@_0N@KHCNHPIB@TestedThread@ 0000000180008008     libresumethrdlst001.obj
 0002:00002018       ??_C@_0BG@EDJJMEFA@Suspend?5threads?5list?6@ 0000000180008018     libresumethrdlst001.obj
 0002:00002030       ??_C@_0DJ@BJHDDPDD@jvmti?9?$DOSuspendThreadList?$CIthread@ 0000000180008030     libresumethrdlst001.obj
 0002:00002070       ??_C@_0BI@NKFHEDBK@Check?5threads?5results?3?6@ 0000000180008070     libresumethrdlst001.obj
 0002:00002088       ??_C@_0BL@MDILKIDM@?5?5?4?4?4?5thread?5?$CD?$CFd?3?5?$CFs?5?$CI?$CFd?$CJ?6@ 0000000180008088     libresumethrdlst001.obj
 0002:000020a8       ??_C@_0L@BOKOKCLN@results?$FLi?$FN@ 00000001800080a8     libresumethrdlst001.obj
 0002:000020b8       ??_C@_0BF@BKLIPBCJ@Resume?5threads?5list?6@ 00000001800080b8     libresumethrdlst001.obj
 0002:000020d0       ??_C@_0DI@KBPIADGM@jvmti?9?$DOResumeThreadList?$CIthreads@ 00000001800080d0     libresumethrdlst001.obj
 0002:00002108       ??_C@_0CC@GOPHFMM@Get?5state?5vector?5for?5each?5threa@ 0000000180008108     libresumethrdlst001.obj
 0002:00002130       ??_C@_0BE@GHIKIJLL@?5?5thread?5?$CD?$CFd?5?$CI?$CFp?$CJ?3?6@ 0000000180008130     libresumethrdlst001.obj
 0002:00002148       ??_C@_0CK@KLKPPJPI@jvmti?9?$DOGetThreadState?$CIthreads?$FLi@ 0000000180008148     libresumethrdlst001.obj
 0002:00002178       ??_C@_0CB@BKACHNJD@?5?5?4?4?4?5got?5state?5vector?3?5?$CFs?5?$CI?$CFd?$CJ@ 0000000180008178     libresumethrdlst001.obj
 0002:000021a0       ??_C@_0FJ@BHKCGJHE@ResumeThreadList?$CI?$CJ?5does?5not?5tur@ 00000001800081a0     libresumethrdlst001.obj
 0002:00002200       ??_C@_0BP@BGBGBECC@Let?5threads?5to?5run?5and?5finish?6@ 0000000180008200     libresumethrdlst001.obj
 0002:00002220       ??_C@_0BL@CLNCJLPF@Wait?5for?5thread?5to?5finish?6@ 0000000180008220     libresumethrdlst001.obj
 0002:00002240       ??_C@_0BL@FOMKIAHJ@Delete?5threads?5references?6@ 0000000180008240     libresumethrdlst001.obj
 0002:00002260       ??_C@_0CB@IPPPCCDL@jni?9?$DODeleteGlobalRef?$CIthreads?$FLi?$FN@ 0000000180008260     libresumethrdlst001.obj
 0002:00002288       ??_C@_0BO@IBGJKPDI@Deallocate?5threads?5array?3?5?$CFp?6@ 0000000180008288     libresumethrdlst001.obj
 0002:000022a8       ??_C@_0CL@NKCGADKC@jvmti?9?$DODeallocate?$CI?$CIunsigned?5cha@ 00000001800082a8     libresumethrdlst001.obj
 0002:000022d8       ??_C@_0BO@BECDNAHN@Deallocate?5results?5array?3?5?$CFp?6@ 00000001800082d8     libresumethrdlst001.obj
 0002:000022f8       ??_C@_0CL@DPBBPFPI@jvmti?9?$DODeallocate?$CI?$CIunsigned?5cha@ 00000001800082f8     libresumethrdlst001.obj
 0002:00002328       ??_C@_0BH@HPEOJMHL@Let?5debugee?5to?5finish?6@ 0000000180008328     libresumethrdlst001.obj
 0002:00002340       ??_C@_0CH@DGAGAHBA@jvmti?9?$DOGetAllThreads?$CI?$CGcount?0?5?$CGt@ 0000000180008340     libresumethrdlst001.obj
 0002:00002368       ??_C@_0CI@BDMNKGJN@jvmti?9?$DOGetThreadInfo?$CIthreads?$FLi?$FN@ 0000000180008368     libresumethrdlst001.obj
 0002:00002390       ??_C@_0CB@IFLPHII@?5?5?4?4?4?5found?5thread?5?$CD?$CFd?3?5?$CFp?5?$CI?$CFs?$CJ@ 0000000180008390     libresumethrdlst001.obj
 0002:000023c0       ??_C@_0FP@JPEOBBIN@Unexpected?5number?5of?5tested?5thr@ 00000001800083c0     libresumethrdlst001.obj
 0002:00002420       ??_C@_0DA@LFMOJOLL@Make?5global?5references?5for?5thre@ 0000000180008420     libresumethrdlst001.obj
 0002:00002450       ??_C@_0EM@DPOEJCND@?$CIfoundThreads?$FLi?$FN?5?$DN?5?$CIjthread?$CJ?5jn@ 0000000180008450     libresumethrdlst001.obj
 0002:000024a0       ??_C@_0BG@DJOPNKEA@?5?5?4?4?4?5thread?5?$CD?$CFd?3?5?$CFp?6@ 00000001800084a0     libresumethrdlst001.obj
 0002:000024b8       ??_C@_0CA@MNKGCBCG@nsk_jvmti_parseOptions?$CIoptions?$CJ@ 00000001800084b8     libresumethrdlst001.obj
 0002:000024d8       ??_C@_07NFPADACG@threads@  00000001800084d8     libresumethrdlst001.obj
 0002:000024e0       ??_C@_0BB@DNEINKNJ@threadsCount?5?$DO?50@ 00000001800084e0     libresumethrdlst001.obj
 0002:000024f8       ??_C@_0DN@MIAMNFPH@?$CIjvmti?5?$DN?5nsk_jvmti_createJVMTIE@ 00000001800084f8     libresumethrdlst001.obj
 0002:00002538       ??_C@_0CF@DFAKMCIB@jvmti?9?$DOAddCapabilities?$CI?$CGsuspend@ 0000000180008538     libresumethrdlst001.obj
 0002:00002560       ??_C@_0CL@PIACJIPK@nsk_jvmti_setAgentProc?$CIagentPro@ 0000000180008560     libresumethrdlst001.obj
 0002:000025a0       ??_C@_1EC@JIJBPKFM@?$AAa?$AAp?$AAi?$AA?9?$AAm?$AAs?$AA?9?$AAw?$AAi?$AAn?$AA?9?$AAc?$AAo?$AAr?$AAe@ 00000001800085a0     MSVCRT:thread_safe_statics.obj
 0002:000025e8       ??_C@_1BK@MGMFAEKH@?$AAk?$AAe?$AAr?$AAn?$AAe?$AAl?$AA3?$AA2?$AA?4?$AAd?$AAl?$AAl@ 00000001800085e8     MSVCRT:thread_safe_statics.obj
 0002:00002608       ??_C@_0BJ@JEBJOJFJ@SleepConditionVariableCS@ 0000000180008608     MSVCRT:thread_safe_statics.obj
 0002:00002628       ??_C@_0BJ@PGPPEPCC@WakeAllConditionVariable@ 0000000180008628     MSVCRT:thread_safe_statics.obj
 0002:00002648       _pDefaultRawDllMain        0000000180008648     MSVCRT:dll_dllmain.obj
 0002:00002648       _pRawDllMain               0000000180008648     MSVCRT:dll_dllmain.obj
 0002:00002650       __xmm@ffffffffffffffffffffffffffffffff 0000000180008650     MSVCRT:utility.obj
 0002:00002660       _load_config_used          0000000180008660     MSVCRT:loadcfg.obj
 0002:00002880       _tls_used                  0000000180008880     MSVCRT:tlssup.obj
 0002:000028a8       __volatile_metadata        00000001800088a8     <linker-defined>
 0002:00002cc0       __rtc_iaa                  0000000180008cc0     MSVCRT:initsect.obj
 0002:00002cc8       __rtc_izz                  0000000180008cc8     MSVCRT:initsect.obj
 0002:00002cd0       __rtc_taa                  0000000180008cd0     MSVCRT:initsect.obj
 0002:00002cd8       __rtc_tzz                  0000000180008cd8     MSVCRT:initsect.obj
 0002:00002ce0       _tls_start                 0000000180008ce0     MSVCRT:tlssup.obj
 0002:00002ce4       _Init_thread_epoch         0000000180008ce4     MSVCRT:thread_safe_statics.obj
 0002:00002ce8       _tls_end                   0000000180008ce8     MSVCRT:tlssup.obj
 0002:000033b8       __IMPORT_DESCRIPTOR_KERNEL32 00000001800093b8     kernel32:KERNEL32.dll
 0002:000033cc       __IMPORT_DESCRIPTOR_VCRUNTIME140 00000001800093cc     vcruntime:VCRUNTIME140.dll
 0002:000033e0       __IMPORT_DESCRIPTOR_api-ms-win-crt-heap-l1-1-0 00000001800093e0     ucrt:api-ms-win-crt-heap-l1-1-0.dll
 0002:000033f4       __IMPORT_DESCRIPTOR_api-ms-win-crt-runtime-l1-1-0 00000001800093f4     ucrt:api-ms-win-crt-runtime-l1-1-0.dll
 0002:00003408       __IMPORT_DESCRIPTOR_api-ms-win-crt-convert-l1-1-0 0000000180009408     ucrt:api-ms-win-crt-convert-l1-1-0.dll
 0002:0000341c       __IMPORT_DESCRIPTOR_api-ms-win-crt-stdio-l1-1-0 000000018000941c     ucrt:api-ms-win-crt-stdio-l1-1-0.dll
 0002:00003430       __IMPORT_DESCRIPTOR_api-ms-win-crt-string-l1-1-0 0000000180009430     ucrt:api-ms-win-crt-string-l1-1-0.dll
 0002:00003444       __NULL_IMPORT_DESCRIPTOR   0000000180009444     kernel32:KERNEL32.dll
 0003:00000030       _Init_global_epoch         000000018000a030     MSVCRT:thread_safe_statics.obj
 0003:00000040       __security_cookie          000000018000a040     MSVCRT:gs_cookie.obj
 0003:00000048       __security_cookie_complement 000000018000a048     MSVCRT:gs_cookie.obj
 0003:00000050       __scrt_native_dllmain_reason 000000018000a050     MSVCRT:utility.obj
 0003:00000058       __isa_available            000000018000a058     MSVCRT:cpu_disp.obj
 0003:0000005c       __isa_enabled              000000018000a05c     MSVCRT:cpu_disp.obj
 0003:00000060       __memset_fast_string_threshold 000000018000a060     MSVCRT:cpu_disp.obj
 0003:00000068       __memset_nt_threshold      000000018000a068     MSVCRT:cpu_disp.obj
 0003:00000070       __scrt_ucrt_dll_is_in_use  000000018000a070     MSVCRT:ucrt_stubs.obj
 0003:00000080       g_wrongHeapCallbacks       000000018000a080     libresumethrdlst001.obj
 0003:00000100       g_szTagInfo                000000018000a100     libresumethrdlst001.obj
 0003:00002040       g_tagFlags                 000000018000c040     libresumethrdlst001.obj
 0003:00002428       g_refsToVerifyCnt          000000018000c428     libresumethrdlst001.obj
 0003:0000242c       g_fakeUserData             000000018000c42c     libresumethrdlst001.obj
 0003:00002430       g_tagVisitCount            000000018000c430     libresumethrdlst001.obj
 0003:000033d0       g_refsToVerify             000000018000d3d0     libresumethrdlst001.obj
 0003:0001aad0       g_userDataError            0000000180024ad0     libresumethrdlst001.obj
 0003:0001ac70       ?_OptionsStorage@?1??__local_stdio_printf_options@@9@4_KA 0000000180024c70     libresumethrdlst001.obj
 0003:0001b368       _tls_index                 0000000180025368     MSVCRT:tlssup.obj
 0003:0001b370       __scrt_current_native_startup_state 0000000180025370     MSVCRT:utility.obj
 0003:0001b378       __scrt_native_startup_lock 0000000180025378     MSVCRT:utility.obj
 0003:0001b3b8       __scrt_debugger_hook_flag  00000001800253b8     MSVCRT:utility_desktop.obj
 0003:0001b3c0       ?__type_info_root_node@@3U__type_info_node@@A 00000001800253c0     MSVCRT:tncleanup.obj
 0003:0001b3d0       ?_OptionsStorage@?1??__local_stdio_scanf_options@@9@4_KA 00000001800253d0     MSVCRT:default_local_stdio_options.obj
 0003:0001b3d8       __favor                    00000001800253d8     MSVCRT:cpu_disp.obj
 0003:0001b3e0       __dyn_tls_init_callback    00000001800253e0     <common>

 entry point at        0001:00003820

 Static symbols

 0000:fffd8000       .debug$S                   0000000180000000     resumethrdlst001.exp
 0000:fffd8000       .debug$S                   0000000180000000     vcruntime:VCRUNTIME140.dll
 0000:fffd8000       .debug$S                   0000000180000000     vcruntime:VCRUNTIME140.dll
 0000:fffd8000       .debug$S                   0000000180000000     vcruntime:VCRUNTIME140.dll
 0000:fffd8000       .debug$S                   0000000180000000     vcruntime:VCRUNTIME140.dll
 0000:fffd8000       .debug$S                   0000000180000000     vcruntime:VCRUNTIME140.dll
 0000:fffd8000       .debug$S                   0000000180000000     vcruntime:VCRUNTIME140.dll
 0000:fffd8000       .debug$S                   0000000180000000     vcruntime:VCRUNTIME140.dll
 0000:fffd8000       .debug$S                   0000000180000000     ucrt:api-ms-win-crt-convert-l1-1-0.dll
 0000:fffd8000       .debug$S                   0000000180000000     ucrt:api-ms-win-crt-heap-l1-1-0.dll
 0000:fffd8000       .debug$S                   0000000180000000     ucrt:api-ms-win-crt-heap-l1-1-0.dll
 0000:fffd8000       .debug$S                   0000000180000000     ucrt:api-ms-win-crt-heap-l1-1-0.dll
 0000:fffd8000       .debug$S                   0000000180000000     ucrt:api-ms-win-crt-heap-l1-1-0.dll
 0000:fffd8000       .debug$S                   0000000180000000     ucrt:api-ms-win-crt-runtime-l1-1-0.dll
 0000:fffd8000       .debug$S                   0000000180000000     ucrt:api-ms-win-crt-runtime-l1-1-0.dll
 0000:fffd8000       .debug$S                   0000000180000000     ucrt:api-ms-win-crt-runtime-l1-1-0.dll
 0000:fffd8000       .debug$S                   0000000180000000     ucrt:api-ms-win-crt-runtime-l1-1-0.dll
 0000:fffd8000       .debug$S                   0000000180000000     ucrt:api-ms-win-crt-runtime-l1-1-0.dll
 0000:fffd8000       .debug$S                   0000000180000000     ucrt:api-ms-win-crt-runtime-l1-1-0.dll
 0000:fffd8000       .debug$S                   0000000180000000     ucrt:api-ms-win-crt-runtime-l1-1-0.dll
 0000:fffd8000       .debug$S                   0000000180000000     ucrt:api-ms-win-crt-runtime-l1-1-0.dll
 0000:fffd8000       .debug$S                   0000000180000000     ucrt:api-ms-win-crt-runtime-l1-1-0.dll
 0000:fffd8000       .debug$S                   0000000180000000     ucrt:api-ms-win-crt-runtime-l1-1-0.dll
 0000:fffd8000       .debug$S                   0000000180000000     ucrt:api-ms-win-crt-runtime-l1-1-0.dll
 0000:fffd8000       .debug$S                   0000000180000000     ucrt:api-ms-win-crt-runtime-l1-1-0.dll
 0000:fffd8000       .debug$S                   0000000180000000     ucrt:api-ms-win-crt-runtime-l1-1-0.dll
 0000:fffd8000       .debug$S                   0000000180000000     ucrt:api-ms-win-crt-runtime-l1-1-0.dll
 0000:fffd8000       .debug$S                   0000000180000000     ucrt:api-ms-win-crt-runtime-l1-1-0.dll
 0000:fffd8000       .debug$S                   0000000180000000     ucrt:api-ms-win-crt-runtime-l1-1-0.dll
 0000:fffd8000       .debug$S                   0000000180000000     ucrt:api-ms-win-crt-stdio-l1-1-0.dll
 0000:fffd8000       .debug$S                   0000000180000000     ucrt:api-ms-win-crt-stdio-l1-1-0.dll
 0000:fffd8000       .debug$S                   0000000180000000     ucrt:api-ms-win-crt-stdio-l1-1-0.dll
 0000:fffd8000       .debug$S                   0000000180000000     ucrt:api-ms-win-crt-stdio-l1-1-0.dll
 0000:fffd8000       .debug$S                   0000000180000000     ucrt:api-ms-win-crt-stdio-l1-1-0.dll
 0000:fffd8000       .debug$S                   0000000180000000     ucrt:api-ms-win-crt-stdio-l1-1-0.dll
 0000:fffd8000       .debug$S                   0000000180000000     ucrt:api-ms-win-crt-stdio-l1-1-0.dll
 0000:fffd8000       .debug$S                   0000000180000000     ucrt:api-ms-win-crt-stdio-l1-1-0.dll
 0000:fffd8000       .debug$S                   0000000180000000     ucrt:api-ms-win-crt-stdio-l1-1-0.dll
 0000:fffd8000       .debug$S                   0000000180000000     ucrt:api-ms-win-crt-stdio-l1-1-0.dll
 0000:fffd8000       .debug$S                   0000000180000000     ucrt:api-ms-win-crt-string-l1-1-0.dll
 0000:fffd8000       .debug$S                   0000000180000000     ucrt:api-ms-win-crt-string-l1-1-0.dll
 0000:fffd8000       .debug$S                   0000000180000000     ucrt:api-ms-win-crt-string-l1-1-0.dll
 0000:fffd8000       .debug$S                   0000000180000000     ucrt:api-ms-win-crt-string-l1-1-0.dll
 0000:fffd8000       .debug$S                   0000000180000000     ucrt:api-ms-win-crt-string-l1-1-0.dll
 0000:fffd8000       .debug$S                   0000000180000000     ucrt:api-ms-win-crt-string-l1-1-0.dll
 0000:fffd8000       .debug$S                   0000000180000000     ucrt:api-ms-win-crt-string-l1-1-0.dll
 0000:fffd8000       .debug$S                   0000000180000000     ucrt:api-ms-win-crt-string-l1-1-0.dll
 0000:fffd8000       .debug$S                   0000000180000000     kernel32:KERNEL32.dll
 0000:fffd8000       .debug$S                   0000000180000000     kernel32:KERNEL32.dll
 0000:fffd8000       .debug$S                   0000000180000000     kernel32:KERNEL32.dll
 0000:fffd8000       .debug$S                   0000000180000000     kernel32:KERNEL32.dll
 0000:fffd8000       .debug$S                   0000000180000000     kernel32:KERNEL32.dll
 0000:fffd8000       .debug$S                   0000000180000000     kernel32:KERNEL32.dll
 0000:fffd8000       .debug$S                   0000000180000000     kernel32:KERNEL32.dll
 0000:fffd8000       .debug$S                   0000000180000000     kernel32:KERNEL32.dll
 0000:fffd8000       .debug$S                   0000000180000000     kernel32:KERNEL32.dll
 0000:fffd8000       .debug$S                   0000000180000000     kernel32:KERNEL32.dll
 0000:fffd8000       .debug$S                   0000000180000000     kernel32:KERNEL32.dll
 0000:fffd8000       .debug$S                   0000000180000000     kernel32:KERNEL32.dll
 0000:fffd8000       .debug$S                   0000000180000000     kernel32:KERNEL32.dll
 0000:fffd8000       .debug$S                   0000000180000000     kernel32:KERNEL32.dll
 0000:fffd8000       .debug$S                   0000000180000000     kernel32:KERNEL32.dll
 0000:fffd8000       .debug$S                   0000000180000000     kernel32:KERNEL32.dll
 0000:fffd8000       .debug$S                   0000000180000000     kernel32:KERNEL32.dll
 0000:fffd8000       .debug$S                   0000000180000000     kernel32:KERNEL32.dll
 0000:fffd8000       .debug$S                   0000000180000000     kernel32:KERNEL32.dll
 0000:fffd8000       .debug$S                   0000000180000000     kernel32:KERNEL32.dll
 0000:fffd8000       .debug$S                   0000000180000000     kernel32:KERNEL32.dll
 0000:fffd8000       .debug$S                   0000000180000000     kernel32:KERNEL32.dll
 0000:fffd8000       .debug$S                   0000000180000000     kernel32:KERNEL32.dll
 0000:fffd8000       .debug$S                   0000000180000000     kernel32:KERNEL32.dll
 0000:fffd8000       .debug$S                   0000000180000000     kernel32:KERNEL32.dll
 0000:fffd8000       .debug$S                   0000000180000000     kernel32:KERNEL32.dll
 0000:fffd8000       .debug$S                   0000000180000000     kernel32:KERNEL32.dll
 0000:fffd8000       .debug$S                   0000000180000000     kernel32:KERNEL32.dll
 0001:00000e74       addRefToVerify             0000000180001e74 f   libresumethrdlst001.obj
 0001:00000ee8       agentProc                  0000000180001ee8 f   libresumethrdlst001.obj
 0001:00001984       agentThreadWrapper         0000000180002984 f   libresumethrdlst001.obj
 0001:00001ad8       check_option               0000000180002ad8 f   libresumethrdlst001.obj
 0001:00001d20       file_basename              0000000180002d20 f   libresumethrdlst001.obj
 0001:00001d50       fillThreadsByName          0000000180002d50 f   libresumethrdlst001.obj
 0001:00002d30       startAgentThreadWrapper    0000000180003d30 f   libresumethrdlst001.obj
 0001:0000305c       syncDebuggeeStatus         000000018000405c f   libresumethrdlst001.obj
 0001:000032e4       capture_previous_context   00000001800042e4 f   MSVCRT:gs_report.obj
 0001:00003358       ?__scrt_initialize_thread_safe_statics@@YAHXZ 0000000180004358 f   MSVCRT:thread_safe_statics.obj
 0001:00003428       ?__scrt_uninitialize_thread_safe_statics@@YAXXZ 0000000180004428 f   MSVCRT:thread_safe_statics.obj
 0001:000034d0       $$000000                   00000001800044d0     MSVCRT:amdsecgs.obj
 0001:00003500       ?dllmain_crt_dispatch@@YAHQEAUHINSTANCE__@@KQEAX@Z 0000000180004500 f   MSVCRT:dll_dllmain.obj
 0001:00003550       ?dllmain_crt_process_attach@@YAHQEAUHINSTANCE__@@QEAX@Z 0000000180004550 f   MSVCRT:dll_dllmain.obj
 0001:00003668       ?dllmain_crt_process_detach@@YAH_N@Z 0000000180004668 f   MSVCRT:dll_dllmain.obj
 0001:000036ec       ?dllmain_dispatch@@YAHQEAUHINSTANCE__@@KQEAX@Z 00000001800046ec f   MSVCRT:dll_dllmain.obj
 0001:00004110       $$000000                   0000000180005110     MSVCRT:guard_dispatch.obj
 0001:00004130       $$000000                   0000000180005130     MSVCRT:guard_xfg_dispatch.obj
 0001:00004146       ?fin$0@?0??dllmain_crt_process_attach@@YAHQEAUHINSTANCE__@@QEAX@Z@4HA 0000000180005146 f   MSVCRT:dll_dllmain.obj
 0001:0000415d       ?fin$0@?0??dllmain_crt_process_detach@@YAH_N@Z@4HA 000000018000515d f   MSVCRT:dll_dllmain.obj
 0001:00004176       ?fin$1@?0??dllmain_crt_process_detach@@YAH_N@Z@4HA 0000000180005176 f   MSVCRT:dll_dllmain.obj
 0001:0000418a       ?filt$0@?0??dllmain_dispatch@@YAHQEAUHINSTANCE__@@KQEAX@Z@4HA 000000018000518a f   MSVCRT:dll_dllmain.obj
 0001:000041c0       __scrt_is_nonwritable_in_current_image$filt$0 00000001800051c0 f   MSVCRT:utility.obj
 0002:00000228       ?__scrt_initialize_tss_var@@3P6AHXZEA 0000000180006228     MSVCRT:thread_safe_statics.obj
 0002:00000350       ?opcLengths@@3QBEB         0000000180006350     libresumethrdlst001.obj
 0002:00002590       GS_ExceptionPointers       0000000180008590     MSVCRT:gs_report.obj
 0002:00002cf0       $unwind$fprintf            0000000180008cf0     libresumethrdlst001.obj
 0002:00002cfc       $unwind$printf             0000000180008cfc     libresumethrdlst001.obj
 0002:00002d08       $unwind$?NewObject@JNIEnv_@@QEAAPEAV_jobject@@PEAV_jclass@@PEAU_jmethodID@@ZZ 0000000180008d08     libresumethrdlst001.obj
 0002:00002d08       $unwind$nsk_lcomplain      0000000180008d08     libresumethrdlst001.obj
 0002:00002d08       $unwind$nsk_ldisplay       0000000180008d08     libresumethrdlst001.obj
 0002:00002d10       $unwind$nsk_lvdisplay      0000000180008d10     libresumethrdlst001.obj
 0002:00002d10       $unwind$_RTC_Initialize    0000000180008d10     MSVCRT:initsect.obj
 0002:00002d10       $unwind$_RTC_Terminate     0000000180008d10     MSVCRT:initsect.obj
 0002:00002d10       $unwind$?__scrt_initialize_thread_safe_statics@@YAHXZ 0000000180008d10     MSVCRT:thread_safe_statics.obj
 0002:00002d1c       $unwind$nsk_complain       0000000180008d1c     libresumethrdlst001.obj
 0002:00002d1c       $unwind$nsk_printf         0000000180008d1c     libresumethrdlst001.obj
 0002:00002d24       $unwind$nsk_lvcomplain     0000000180008d24     libresumethrdlst001.obj
 0002:00002d3c       $unwind$nsk_ltrace         0000000180008d3c     libresumethrdlst001.obj
 0002:00002d3c       $unwind$__report_gsfailure 0000000180008d3c     MSVCRT:gs_report.obj
 0002:00002d44       $unwind$nsk_lvtrace        0000000180008d44     libresumethrdlst001.obj
 0002:00002d44       $unwind$__raise_securityfailure 0000000180008d44     MSVCRT:gs_report.obj
 0002:00002d44       $unwind$__scrt_initialize_crt 0000000180008d44     MSVCRT:utility.obj
 0002:00002d44       $unwind$__scrt_initialize_onexit_tables 0000000180008d44     MSVCRT:utility.obj
 0002:00002d44       $unwind$__scrt_release_startup_lock 0000000180008d44     MSVCRT:utility.obj
 0002:00002d44       $unwind$__scrt_uninitialize_crt 0000000180008d44     MSVCRT:utility.obj
 0002:00002d44       $unwind$_onexit            0000000180008d44     MSVCRT:utility.obj
 0002:00002d4c       $unwind$nsk_lverify        0000000180008d4c     libresumethrdlst001.obj
 0002:00002d5c       $unwind$nsk_vprintf        0000000180008d5c     libresumethrdlst001.obj
 0002:00002d6c       $unwind$?nsk_jni_lverify@@YAHHPEAUJNIEnv_@@HQEBDH1ZZ 0000000180008d6c     libresumethrdlst001.obj
 0002:00002d80       $unwind$?nsk_jni_check_exception@@YAHPEAUJNIEnv_@@QEBDH@Z 0000000180008d80     libresumethrdlst001.obj
 0002:00002d9c       $unwind$nsk_jvmti_parseOptions 0000000180008d9c     libresumethrdlst001.obj
 0002:00002db8       $unwind$nsk_jvmti_createJVMTIEnv 0000000180008db8     libresumethrdlst001.obj
 0002:00002dcc       $unwind$check_option       0000000180008dcc     libresumethrdlst001.obj
 0002:00002dcc       $unwind$nsk_jvmti_findOptionValue 0000000180008dcc     libresumethrdlst001.obj
 0002:00002dcc       $unwind$nsk_jvmti_waitForSync 0000000180008dcc     libresumethrdlst001.obj
 0002:00002dcc       $unwind$_DllMainCRTStartup 0000000180008dcc     MSVCRT:dll_dllmain.obj
 0002:00002ddc       $unwind$Java_nsk_jvmti_unit_FollowReferences_FollowRefObjects_resetTags 0000000180008ddc     libresumethrdlst001.obj
 0002:00002ddc       $unwind$addRefToVerify     0000000180008ddc     libresumethrdlst001.obj
 0002:00002ddc       $unwind$nsk_jvmti_resetAgentData 0000000180008ddc     libresumethrdlst001.obj
 0002:00002ddc       $unwind$nsk_jvmti_resumeSync 0000000180008ddc     libresumethrdlst001.obj
 0002:00002ddc       $unwind$__scrt_initialize_default_local_stdio_options 0000000180008ddc     MSVCRT:default_local_stdio_options.obj
 0002:00002ddc       $unwind$?dllmain_crt_dispatch@@YAHQEAUHINSTANCE__@@KQEAX@Z 0000000180008ddc     MSVCRT:dll_dllmain.obj
 0002:00002ddc       $unwind$DllMain            0000000180008ddc     MSVCRT:dll_dllmain_stub.obj
 0002:00002ddc       $unwind$__GSHandlerCheck   0000000180008ddc     MSVCRT:gshandler.obj
 0002:00002ddc       $unwind$?__scrt_uninitialize_thread_safe_statics@@YAXXZ 0000000180008ddc     MSVCRT:thread_safe_statics.obj
 0002:00002ddc       $unwind$__scrt_acquire_startup_lock 0000000180008ddc     MSVCRT:utility.obj
 0002:00002ddc       $unwind$__scrt_dllmain_after_initialize_c 0000000180008ddc     MSVCRT:utility.obj
 0002:00002ddc       $unwind$__scrt_dllmain_before_initialize_c 0000000180008ddc     MSVCRT:utility.obj
 0002:00002ddc       $unwind$__scrt_dllmain_crt_thread_attach 0000000180008ddc     MSVCRT:utility.obj
 0002:00002ddc       $unwind$__scrt_dllmain_crt_thread_detach 0000000180008ddc     MSVCRT:utility.obj
 0002:00002ddc       $unwind$__scrt_dllmain_uninitialize_c 0000000180008ddc     MSVCRT:utility.obj
 0002:00002ddc       $unwind$__scrt_dllmain_uninitialize_critical 0000000180008ddc     MSVCRT:utility.obj
 0002:00002ddc       $unwind$atexit             0000000180008ddc     MSVCRT:utility.obj
 0002:00002de4       $unwind$nsk_jvmti_findOptionIntValue 0000000180008de4     libresumethrdlst001.obj
 0002:00002df4       $unwind$nsk_jvmti_lverify  0000000180008df4     libresumethrdlst001.obj
 0002:00002e08       $unwind$exitOnError        0000000180008e08     libresumethrdlst001.obj
 0002:00002e18       $unwind$Java_nsk_share_jvmti_ArgumentHandler_getAgentOptionsString 0000000180008e18     libresumethrdlst001.obj
 0002:00002e2c       $unwind$Java_nsk_jvmti_unit_FollowReferences_FollowRefObjects_getTag 0000000180008e2c     libresumethrdlst001.obj
 0002:00002e2c       $unwind$Java_nsk_share_jvmti_DebugeeClass_checkStatus 0000000180008e2c     libresumethrdlst001.obj
 0002:00002e2c       $unwind$agentThreadWrapper 0000000180008e2c     libresumethrdlst001.obj
 0002:00002e3c       $unwind$startAgentThreadWrapper 0000000180008e3c     libresumethrdlst001.obj
 0002:00002e58       $unwind$syncDebuggeeStatus 0000000180008e58     libresumethrdlst001.obj
 0002:00002e58       $unwind$__scrt_dllmain_exception_filter 0000000180008e58     MSVCRT:utility.obj
 0002:00002e6c       $unwind$Java_nsk_share_jvmti_DebugeeClass_resetAgentData 0000000180008e6c     libresumethrdlst001.obj
 0002:00002e74       $unwind$MA_checkStatus     0000000180008e74     libresumethrdlst001.obj
 0002:00002e88       $unwind$Java_nsk_jvmti_unit_FollowReferences_FollowRefObjects_setTag 0000000180008e88     libresumethrdlst001.obj
 0002:00002ea0       $unwind$Java_nsk_jvmti_unit_FollowReferences_FollowRefObjects_addRefToVerify 0000000180008ea0     libresumethrdlst001.obj
 0002:00002ebc       $unwind$Agent_Initialize   0000000180008ebc     libresumethrdlst001.obj
 0002:00002edc       $unwind$fillThreadsByName  0000000180008edc     libresumethrdlst001.obj
 0002:00002ef4       $unwind$agentProc          0000000180008ef4     libresumethrdlst001.obj
 0002:00002f0c       $unwind$capture_previous_context 0000000180008f0c     MSVCRT:gs_report.obj
 0002:00002f18       $unwind$__GSHandlerCheckCommon 0000000180008f18     MSVCRT:gshandler.obj
 0002:00002f20       $xdatasym                  0000000180008f20     MSVCRT:amdsecgs.obj
 0002:00002f24       $unwind$?dllmain_crt_process_attach@@YAHQEAUHINSTANCE__@@QEAX@Z 0000000180008f24     MSVCRT:dll_dllmain.obj
 0002:00002f60       $unwind$?fin$0@?0??dllmain_crt_process_attach@@YAHQEAUHINSTANCE__@@QEAX@Z@4HA 0000000180008f60     MSVCRT:dll_dllmain.obj
 0002:00002f60       $unwind$?fin$0@?0??dllmain_crt_process_detach@@YAH_N@Z@4HA 0000000180008f60     MSVCRT:dll_dllmain.obj
 0002:00002f60       $unwind$?fin$1@?0??dllmain_crt_process_detach@@YAH_N@Z@4HA 0000000180008f60     MSVCRT:dll_dllmain.obj
 0002:00002f68       $unwind$?dllmain_crt_process_detach@@YAH_N@Z 0000000180008f68     MSVCRT:dll_dllmain.obj
 0002:00002fbc       $unwind$?dllmain_dispatch@@YAHQEAUHINSTANCE__@@KQEAX@Z 0000000180008fbc     MSVCRT:dll_dllmain.obj
 0002:00002fe4       $unwind$?filt$0@?0??dllmain_dispatch@@YAHQEAUHINSTANCE__@@KQEAX@Z@4HA 0000000180008fe4     MSVCRT:dll_dllmain.obj
 0002:00002fec       $unwind$__scrt_is_nonwritable_in_current_image 0000000180008fec     MSVCRT:utility.obj
 0002:0000300c       $unwind$__scrt_is_nonwritable_in_current_image$filt$0 000000018000900c     MSVCRT:utility.obj
 0002:00003014       $unwind$__scrt_fastfail    0000000180009014     MSVCRT:utility_desktop.obj
 0002:00003024       $unwind$__security_init_cookie 0000000180009024     MSVCRT:gs_support.obj
 0002:00003030       $unwind$__isa_available_init 0000000180009030     MSVCRT:cpu_disp.obj
 0002:00003040       $xdatasym                  0000000180009040     MSVCRT:guard_dispatch.obj
 0002:00003048       $xdatasym                  0000000180009048     MSVCRT:guard_xfg_dispatch.obj
 0002:00003050       .edata                     0000000180009050     resumethrdlst001.exp
 0002:00003078       rgpv                       0000000180009078     resumethrdlst001.exp
 0002:000030b0       rgszName                   00000001800090b0     resumethrdlst001.exp
 0002:000030e8       rgwOrd                     00000001800090e8     resumethrdlst001.exp
 0002:00003104       szName                     0000000180009104     resumethrdlst001.exp
 0002:00003119       $N00001                    0000000180009119     resumethrdlst001.exp
 0002:00003128       $N00002                    0000000180009128     resumethrdlst001.exp
 0002:00003135       $N00003                    0000000180009135     resumethrdlst001.exp
 0002:0000317a       $N00004                    000000018000917a     resumethrdlst001.exp
 0002:000031b7       $N00005                    00000001800091b7     resumethrdlst001.exp
 0002:000031ff       $N00006                    00000001800091ff     resumethrdlst001.exp
 0002:0000323f       $N00007                    000000018000923f     resumethrdlst001.exp
 0002:0000327c       $N00008                    000000018000927c     resumethrdlst001.exp
 0002:000032b7       $N00009                    00000001800092b7     resumethrdlst001.exp
 0002:000032e5       $N00010                    00000001800092e5     resumethrdlst001.exp
 0002:00003316       $N00011                    0000000180009316     resumethrdlst001.exp
 0002:00003345       $N00012                    0000000180009345     resumethrdlst001.exp
 0002:00003374       $N00013                    0000000180009374     resumethrdlst001.exp
 0002:000033a9       $N00014                    00000001800093a9     resumethrdlst001.exp
 0002:0000381a       .idata$6                   000000018000981a     kernel32:KERNEL32.dll
 0002:0000387e       .idata$6                   000000018000987e     vcruntime:VCRUNTIME140.dll
 0002:00003a24       .idata$6                   0000000180009a24     ucrt:api-ms-win-crt-heap-l1-1-0.dll
 0002:00003a44       .idata$6                   0000000180009a44     ucrt:api-ms-win-crt-runtime-l1-1-0.dll
 0002:00003a66       .idata$6                   0000000180009a66     ucrt:api-ms-win-crt-convert-l1-1-0.dll
 0002:00003a88       .idata$6                   0000000180009a88     ucrt:api-ms-win-crt-stdio-l1-1-0.dll
 0002:00003aa8       .idata$6                   0000000180009aa8     ucrt:api-ms-win-crt-string-l1-1-0.dll
 0003:00000000       ?codeAttributeName@@3PEBDEB 000000018000a000     libresumethrdlst001.obj
 0003:00000008       ?lineNumberAttributeName@@3PEBDEB 000000018000a008     libresumethrdlst001.obj
 0003:00000010       ?localVarAttributeName@@3PEBDEB 000000018000a010     libresumethrdlst001.obj
 0003:00000018       ?localVarTypeAttributeName@@3PEBDEB 000000018000a018     libresumethrdlst001.obj
 0003:00000020       ?stackMapAttributeName@@3PEBDEB 000000018000a020     libresumethrdlst001.obj
 0003:00000028       ?callBytes@@3PAEA          000000018000a028     libresumethrdlst001.obj
 0003:0000002c       ?allocBytes@@3PAEA         000000018000a02c     libresumethrdlst001.obj
 0003:0001aad4       redefineAttempted          0000000180024ad4     libresumethrdlst001.obj
 0003:0001aad8       nsk_context                0000000180024ad8     libresumethrdlst001.obj
 0003:0001aae4       redefineSucceed            0000000180024ae4     libresumethrdlst001.obj
 0003:0001aae8       agentFailed                0000000180024ae8     libresumethrdlst001.obj
 0003:0001aaec       currentAgentStatus         0000000180024aec     libresumethrdlst001.obj
 0003:0001aaf0       context                    0000000180024af0     libresumethrdlst001.obj
 0003:0001aba8       agentThread                0000000180024ba8     libresumethrdlst001.obj
 0003:0001abb0       agentThreadProc            0000000180024bb0     libresumethrdlst001.obj
 0003:0001abb8       agentThreadArg             0000000180024bb8     libresumethrdlst001.obj
 0003:0001abc0       agent_data                 0000000180024bc0     libresumethrdlst001.obj
 0003:0001abd0       jvmti_env                  0000000180024bd0     libresumethrdlst001.obj
 0003:0001abd8       jvm                        0000000180024bd8     libresumethrdlst001.obj
 0003:0001abe0       jni_env                    0000000180024be0     libresumethrdlst001.obj
 0003:0001abe8       checkStatus_func           0000000180024be8     libresumethrdlst001.obj
 0003:0001abf0       ?codeAttributeIndex@@3GA   0000000180024bf0     libresumethrdlst001.obj
 0003:0001abf4       ?lineNumberAttributeIndex@@3GA 0000000180024bf4     libresumethrdlst001.obj
 0003:0001abf8       ?localVarAttributeIndex@@3GA 0000000180024bf8     libresumethrdlst001.obj
 0003:0001abfc       ?localVarTypeAttributeIndex@@3GA 0000000180024bfc     libresumethrdlst001.obj
 0003:0001ac00       ?stackMapAttributeIndex@@3GA 0000000180024c00     libresumethrdlst001.obj
 0003:0001ac04       ?stackFrameOffset@@3GA     0000000180024c04     libresumethrdlst001.obj
 0003:0001ac08       ?mode@@3HA                 0000000180024c08     libresumethrdlst001.obj
 0003:0001ac0c       ?constantPoolSize@@3GA     0000000180024c0c     libresumethrdlst001.obj
 0003:0001ac10       ?orig@@3PEBEEB             0000000180024c10     libresumethrdlst001.obj
 0003:0001ac18       ?gen@@3PEAEEA              0000000180024c18     libresumethrdlst001.obj
 0003:0001ac20       ?inputPos@@3PEAEEA         0000000180024c20     libresumethrdlst001.obj
 0003:0001ac28       ?endPos@@3PEBEEB           0000000180024c28     libresumethrdlst001.obj
 0003:0001ac30       ?genPos@@3PEAEEA           0000000180024c30     libresumethrdlst001.obj
 0003:0001ac38       ?markPos@@3PEAEEA          0000000180024c38     libresumethrdlst001.obj
 0003:0001ac40       ?constantPool@@3PEAPEADEA  0000000180024c40     libresumethrdlst001.obj
 0003:0001ac48       ?constantPoolCount@@3GA    0000000180024c48     libresumethrdlst001.obj
 0003:0001ac4c       ?zeroBytes@@3PAEA          0000000180024c4c     libresumethrdlst001.obj
 0003:0001ac50       ?codeLength@@3IA           0000000180024c50     libresumethrdlst001.obj
 0003:0001ac54       threadsCount               0000000180024c54     libresumethrdlst001.obj
 0003:0001ac58       ?map@@3PEAIEA              0000000180024c58     libresumethrdlst001.obj
 0003:0001ac60       ?widening@@3PEACEA         0000000180024c60     libresumethrdlst001.obj
 0003:0001ac68       timeout                    0000000180024c68     libresumethrdlst001.obj
 0003:0001ac80       ?str@?1??TranslateState@@YAPEBDH@Z@4PADA 0000000180024c80     libresumethrdlst001.obj
 0003:0001adb0       GS_ExceptionRecord         0000000180024db0     MSVCRT:gs_report.obj
 0003:0001ae50       GS_ContextRecord           0000000180024e50     MSVCRT:gs_report.obj
 0003:0001b320       ?g_tss_cv@@3U_RTL_CONDITION_VARIABLE@@A 0000000180025320     MSVCRT:thread_safe_statics.obj
 0003:0001b328       ?g_tss_event@@3PEAXEA      0000000180025328     MSVCRT:thread_safe_statics.obj
 0003:0001b330       ?g_tss_mutex@@3U_RTL_CRITICAL_SECTION@@A 0000000180025330     MSVCRT:thread_safe_statics.obj
 0003:0001b358       ?g_sleep_condition_variable_cs@@3P6AHPEAU_RTL_CONDITION_VARIABLE@@PEAU_RTL_CRITICAL_SECTION@@K@ZEA 0000000180025358     MSVCRT:thread_safe_statics.obj
 0003:0001b360       ?g_wake_all_condition_variable@@3P6AXPEAU_RTL_CONDITION_VARIABLE@@@ZEA 0000000180025360     MSVCRT:thread_safe_statics.obj
 0003:0001b36c       ?__proc_attached@@3HA      000000018002536c     MSVCRT:dll_dllmain.obj
 0003:0001b380       ?is_initialized_as_dll@@3_NA 0000000180025380     MSVCRT:utility.obj
 0003:0001b381       ?module_local_atexit_table_initialized@@3_NA 0000000180025381     MSVCRT:utility.obj
 0003:0001b388       ?module_local_atexit_table@@3U_onexit_table_t@@A 0000000180025388     MSVCRT:utility.obj
 0003:0001b3a0       ?module_local_at_quick_exit_table@@3U_onexit_table_t@@A 00000001800253a0     MSVCRT:utility.obj
